:020000041100E9
:10300000002373B52B4D2C4C28006361022601F080
:103010006BF94021FE2221742800284B009601F014
:10302000B5F9002836D1217CFF222800244B0096D8
:1030300001F0ACF900282DD1224BA2899A4226D169
:10304000E389214A93420DD1204B6361204B2268D2
:10305000002A03D1002B01D043CB43C4280001F048
:1030600081F973BD1B4A934201D00023EFE71A4B4D
:103070001A4A1B68934206D9C02304222800217CE7
:103080009B0001F0F9F9114B6361154BDFE7002359
:103090002374EAE7CC233821AC2228009B01217459
:1030A00001F0EAF90028F2D10E4B63610E4BE38187
:1030B0000E4BCCE7D441FF1FA061FF1FAC61FF1F87
:1030C000AE61FF1F59590000830500001541001132
:1030D00004BD001182150000C461FF1F87130000AA
:1030E00010BD0011CD410011AAAAFFFFF8BC0011CC
:1030F000F7B5164B0192C318021D002000938823D8
:103100005B05D3181B685C1C1AD09CB2402C18D8E5
:103110008D781E0CAC466746CD782D023D43AE42FD
:1031200006D1019800280ED110000C70240A4C70B2
:1031300003249BB20733A343D218009B9A42DED3E9
:10314000FEBD4432F9E71000FAE7C046FC0F00006C
:10315000802213B503000324019189B25201073183
:103160009B18A14304305A1A88235B05C3181B68B7
:10317000591C03D190429241104016BD99B240298A
:1031800007D80B000733A343C0189042ECD30020AC
:10319000F3E74430F9E7134B134A1B68126810B584
:1031A000FA24934201D81A00F824104BE4021B6859
:1031B0009A4210D813000E4A12689A420ED3013375
:1031C00007D1F823DB029C4203D10A49054808F0E5
:1031D000EFFA200010BDFC24E402ECE7FE24E40238
:1031E000F7E7C04600C0071100D0071100E0071143
:1031F00000F00711FFFFFF7FF0B59BB015000490B2
:103200000391402A00D9A0E006AB59801A80FFF74D
:10321000C2FF0400042816D9002206A9FFF768FFA0
:10322000052810D906AB1B88AB420CD1002D07D066
:10323000514B2A000499C01808F0CAFC002802D19A
:1032400001201BB0F0BD06AB1D8020000699FFF7E2
:103250007FFF041E7BD1069B0793FFF79CFF802313
:103260005B01C618802307001B039E4201D3F8268A
:10327000F60288235B05F31801931B68013302D023
:10328000019808F01DFB3D49019808F091FA3B1D9B
:103290000293331D05938822029B52059B181B68DD
:1032A00008935A1C3CD044219AB20091402A04D879
:1032B0000320D11D814389B2009103991B0C8B42DD
:1032C00024D0402A22D80122300008A9FFF710FF9D
:1032D000021E1BD1380008A9FFF70AFF04000428CA
:1032E00031D9009A059B9B1880225201B218934253
:1032F00040D288235B05C118009A09A808F0C0FBDA
:103300001D4B009A09A9F01808F0D2FB009A029B05
:103310009446634402931A4B029AFB189A42BAD31A
:1033200088235B05FC1821680198013908F040FAF0
:10333000200008F0C5FA039A07AB5A8030000799BD
:10334000FFF706FF0400002C03D1002079E70428D2
:10335000FBD988235B05E018069908F029FA0323B6
:10336000EA1C9A4300D16BE7034B0499E01808F07C
:103370009FFB65E70424ECE704000011FFFFFF7FDB
:10338000F80F0000F7B505001400402A21D80027E7
:1033900001AE71803780FFF7FEFE042816D93A008F
:1033A0003100FFF7A5FE042810D93688BC420BD0A7
:1033B000BD4209D0221CB44200D9321C064B92B245
:1033C000C118280008F05CFB30B2FEBDC04300B25B
:1033D000FBE703204042F8E70400001137B5042260
:1033E00004000D0001A81649FFF7CCFF02000428D5
:1033F0000BD1019BA34208D3AB4204D0104901A8D2
:103400000195FFF7F9FE01203EBD0E4C2368200018
:10341000019308F055FA019920000139019108F053
:10342000C7F980235B01E418074B9C42EED10422CC
:10343000034901A80195FFF7DFFE0020E4E7C0463D
:103440005555000000C007110000081130B589B0C3
:1034500008F056FA10226946254808F081F9254BF4
:10346000009A9A420ED1019B029A0F2B33D8002169
:1034700001240698013B08D2002900D00292029B49
:10348000013331D10023029325E0551CF2D1020013
:103490002100EFE710341022200004A908F060F9A1
:1034A000029B013301D1069B0293882304995B059B
:1034B000C918059B06981A03120B049105928142C4
:1034C00003D02B4201D108F0DBFA019B013B0193B1
:1034D000019B002BDED1029B002B03D004930498A8
:1034E0004168084709B030BDE025014C2D03EFE7E6
:1034F00000000111504859368022F8B5964C974B80
:10350000D200002120001C6008F012FB2300944A26
:1035100088331A60934B1A786A23002A00D011333B
:10352000E3620A232365904B37221B780820A363AC
:103530008E4B2118E361102323628D4B3B25636181
:10354000C823DB00A36123008C331A602823013ACF
:10355000E26320646364CA67043A211DCA672100DC
:10356000BC310D602100C03108602100C4310B6006
:1035700021000635CC310D602100083DC8310D60B9
:103580002100D0310A602200D43210602200D832EB
:10359000136022000227E032210017604222DC3152
:1035A0000A6021001B3DE4310D602100E831086014
:1035B0002100EC310B6023000521F4331960230056
:1035C000F0331A602300183290331A6023009433CA
:1035D000186023001E3A98331A60AF23DB00236083
:1035E000644BFA262363644B644DE360644BF03113
:1035F000A3642300FF31FC33B600A16021611E608B
:10360000A5627325E5656D3D6565A56596255D4AF1
:10361000AD00E264666258606766A566002709250A
:10362000A767E566584F594D606720002567E26738
:103630003A6015279C30676007001A203860200028
:10364000A0300700212038602000A83007004C4837
:1036500038602000F830066026006427A436376002
:1036600026005F3FAC3637602600033FB036376038
:103670002600C637B436376026000027B8363760D4
:1036800038269E60424E96205E64424E5A66DE6147
:10369000414E9A645E62F53EFF3E9E621E269A6728
:1036A000354A8000DE661F675F67DD651D6618624C
:1036B000DA67BE23394A5B00E250394BD8382350D1
:1036C00004302250C4225200A350C623E4205B00E1
:1036D000E1500433334AE1503349344BD16034492B
:1036E000800019503349E938FF3819503249043005
:1036F000195032493248D16132491163324951631C
:103700001900F4310860CE20304940001160304982
:10371000195019002F48F83108602F49D1658221CE
:103720002E4A89005A501A002D490832D1671A00D2
:103730002C49B432116088212B4A89005A501A0052
:103740002A49883211602A4ADA6408F019F80120FF
:1037500008F09EF9F8BDC0460004FF1F4464FF1F37
:10376000106FFF1F1044FF1F4A0AFF1F3A07000097
:1037700080C3C9019A020000DC0500006A1800003D
:1037800050C3000088130000F009FF1F204E000006
:103790006509FF1F68100000C409000040420F00C7
:1037A00010270000FC00FF1F791CFF1F0000FF1FF7
:1037B000CD2CFF1F5530FF1FED2EFF1F3920FF1F9F
:1037C0002927FF1F5520FF1F0122FF1FC51FFF1FB5
:1037D0004D29FF1F352AFF1F9119FF1F5928FF1F71
:1037E0007D25FF1F8925FF1FC51EFF1F7D1FFF1F92
:1037F0003D1EFF1F0223F0B50124604D604E2B706B
:10380000604B91B01C70604F03933368002120001F
:10381000FB7006F0E9FD200006F0E0FC0023984272
:1038200005D0FA78552A02D0332A00D099E03360C7
:10383000042006F041FF07F0D3FFFFF75DFE08F01C
:103840002FF91F2201240021504B10AE1A70504B4B
:103850001C70504B1970504B19689143163A0A432B
:103860001A60602219689143403A0A431A6008F0CE
:1038700077F907F0FDFE494B9847C120FF21484BDF
:1038800080001A588A431A50C522920098588843DB
:10389000BF39014399509858424908408021C901D5
:1038A0000143802099509958C0050902090A014333
:1038B000995080213C48490107F042FF0323220030
:1038C0003A49019400933A4807F0AAFE2C2239495C
:1038D00005A808F0D5F805AC61782078023406F028
:1038E0009DFCA642F8D1344C344B226803201A4088
:1038F000A023DB0213432360802322689B0413432D
:10390000236022682E4B1A4080239B0313432360BD
:103910002C4A2D4B934200D8012008F069F908F099
:10392000E7F880232268DB0413432360287807F03C
:10393000FFFF039B1878C0B208F022F808F0C0F827
:103940002249042008F014F806F082FE00F040F846
:1039500000F0E8FD00F090FE00F00AFA002011B03F
:10396000F0BD00932100194A042007F091FF802345
:10397000DB059C62FFF76AFD5AE7C0464A0AFF1F53
:1039800034F000401044FF1FD061FF1F480AFF1FA2
:10399000490AFF1F680AFF1FBCF00040E1A20000B7
:1039A00000E100E0FF00FFFF1444FF1F9856FF1FD7
:1039B0001454FF1F20BC001114F00040FF7FF8FFDB
:1039C000FFFF9FFF0080FF1F106FFF1F3B000108DC
:1039D000002210B51100112007F03AFF10BD0000C1
:1039E000F8B500230926364F364C3B62E3681120B8
:1039F000B343E36008F06CF8112007F079FE112062
:103A000007F0D6FF4023226810251343236080234C
:103A10006268DB02134363608023A26802211343C0
:103A2000A360A368284A08201340A3608023A268EB
:103A30009B0113430122A360236CAB432364236CDB
:103A40001343236480231B013B62226B1F4B1A40EC
:103A50002263626B1A406263A26B1A40A263E26B3C
:103A60001340E363E3681A4A1340E36006F0D6FBB1
:103A70000121082006F0E6FC8023164A5B00516C09
:103A800011200B43536407F0D3FEFD21C720124BD6
:103A9000124A89005A50A36B80002B43A363E3684A
:103AA0000F4A3343E3600F4B195811408022120232
:103AB0000A431A50802292051A600B4B5D63F8BDD1
:103AC00000F000403CF00040FFFFDFFFEFFFEFFFA2
:103AD000FFFF7FFF003800400000FF1F5118FF1F4D
:103AE000FF00FFFF00E100E00000054070B5284C3A
:103AF000238C002B23D0228A002A21D1DA002382B2
:103B00006382A382E38223836383A383E3832260AC
:103B10006260A260E2601F4D1F4A6420EB80934206
:103B20000AD8FA220020D200934205D91B4A0A2162
:103B3000981807F045FDC0B200232872238470BD99
:103B40000720E11CCA7F01320240CA7705D1032554
:103B5000201DC17F01312940C17708325200A35294
:103B6000002321001A00088A01321B180231082A9A
:103B7000F9D1221DD27F9200A350626823689B185E
:103B8000A2689B18E2689B185B099BB2C3E7C0461A
:103B90001061FF1FB861FF1FB70B000030F8FFFF77
:103BA00030B503A804880B20002C0ED14968074DBE
:103BB00008784978090201430A20A94205D1012168
:103BC00020001980024B1B7A137030BD192A0000A7
:103BD000B861FF1FF7B5150008AA16884A680F4F8D
:103BE00014785278120222430A24BA4214D10122D4
:103BF000DBB2019200962A0007F07AFC041E0BD17A
:103C0000074B1B68002B07D068782A780002104306
:103C100042425041013098472000FEBD0229000079
:103C20003C61FF1F30B5012503790400BFB02B4272
:103C300011D00A49408806F0C7FF28420BD0084B34
:103C400001A95B8D4D800B80064B00221B7A60889A
:103C50000B7104F0ABF83FB030BDC0463461FF1FBC
:103C60004840FF1FB861FF1F10B50549054806F021
:103C700061FF0421044A054806F01EFF10BDC0463E
:103C80003461FF1FFFFF00004CBC00114840FF1FC4
:103C900010B5024804F00CFF10BDC046253C0011D1
:103CA000012303700B4B1A7A4270022282709A78B9
:103CB000C270DA780271032242711A7982715A79DC
:103CC000C2710C2202729A794272DB7983720B20E4
:103CD0007047C046B861FF1F022310B50370013B57
:103CE00043700533837010330371443B43712A33AF
:103CF00083714433C37100230372064B04001B8895
:103D000043720A30FFF7CCFF831D0A30C0B2E37064
:103D100010BDC046B861FF1F10B5142007F0C8FCE5
:103D2000124B14220021186007F002FF002007F058
:103D3000C7FC012007F044FE022007F081FD0320AC
:103D400004F05AF9042006F06FF9052003F098FBFF
:103D5000062004F065F8072001F062FA082006F05A
:103D60008BFE092001F03CF810BDC0464061FF1FEA
:103D700007F03EFE012007F063FE07F059FE000049
:103D8000094B10B50400984205D0012904D1200048
:103D9000064906F0CFFE10BD0229FCD1013904F01E
:103DA00045FE0028F3D0F6E7FEFF00006661FF1F26
:103DB00070B50D7A100004AA2C0016881022144049
:103DC000154220D1002E20D10A78022A18D14A6843
:103DD000517815780E4A09022943914205D00D4ABF
:103DE000914209D01C800A2404E014220A491A8056
:103DF00007F046FE200070BD0C2208491A80F7E744
:103E00001C800124F6E70824F4E70B24F2E7C046FF
:103E1000F3FF0000F4FF00009C42FF1F28BD0011CB
:103E200010B504000749084806F084FE074804F06E
:103E30007FFD0020E40704D50721054A054806F068
:103E40003BFE10BD6661FF1FFFFF0000813D0011BA
:103E500090BC00118C40FF1F00B50C4BBFB01A780E
:103E60000B4902A800F0C2FC6B4680B2D880002843
:103E700009D06A46074B01A91B889380064B002294
:103E8000188803F093FF3FB000BDC0464461FF1F98
:103E90004561FF1FE640FF1FF041FF1F00B50C4BBF
:103EA000BFB01A780B4902A801F0C6FE6B4680B27B
:103EB000D880002809D06A46074B01A95B8D938002
:103EC000064B0022188803F071FF3FB000BDC046CA
:103ED0006E61FF1F6F61FF1F8C40FF1FF041FF1FCE
:103EE000F7B50E00377A1C0008AB11003D001A88A8
:103EF00020231D401F423CD13378022B3BD17368F5
:103F00001F785B781B023B431E4FBB4208D01E4FFD
:103F1000BB4214D01D4DAB4221D00A252800FEBD66
:103F2000002A2AD1142C2AD82200F06807F0A8FD14
:103F3000174B1C70012CF1D9FFF7B0FFEEE7002AF8
:103F40001BD1202C1BD82200F06807F099FD114BE3
:103F500004211C70104B187807F04AFCDEE7E3B22E
:103F60000124009201940A00310007F0C1FA050013
:103F7000D4E70825D2E70125D0E70B25CEE70D25AC
:103F8000CCE7C046F3FF0000F4FF00000229000068
:103F90006E61FF1F4461FF1FF061FF1F332310B5E7
:103FA000040003700A220749013007F069FD064B3F
:103FB0000F201B681A0AE37222731A0C1B0E62731D
:103FC000A37310BDB861FF1FE061FF1F30B501256D
:103FD00003790400BFB02B4213D00B49408806F090
:103FE000F3FD28420DD06A46084B02A81B88938037
:103FF000FFF7D4FF6B46D8800022608801A903F048
:10400000D5FE3FB030BDC0466661FF1FE640FF1FD2
:1040100010B5024804F04CFD10BDC046CD3F001164
:1040200070B5160004AA148805AA15784A68507855
:10403000117800022A4A0843801805284BD807F057
:104040009FFD03131E29343F0720032C0BD80422A5
:10405000121BAA4200D92A0022491A8030000919ED
:1040600007F00EFD002070BD0720112CFBD8122296
:10407000121BAA4200D92A001B491A80EEE707202A
:104080000E2CF0D80F22121BAA4200D92A00174981
:104090001A80E3E70720032CE5D80422121BAA426A
:1040A00000D92A0012491A80D8E70720032CDAD851
:1040B0000422121BAA4200D92A000E491A80CDE719
:1040C0000720032CCFD80422121BAA4200D92A00B1
:1040D00009491A80C2E700220A201A80C3E7C046B5
:1040E000DCD5FFFFDBBC00118C61FF1FCBBC0011D6
:1040F000C6BC0011C1BC0011BCBC001110B50D2123
:10410000024A034806F0D8FC10BDC046B0BC0011FE
:10411000FC40FF1FF0B50024274E85B03000B4717D
:1041200000F0E2F8254D264BEA89297C9A422FD1EE
:104130000423300003AA00F057F90400300000F017
:1041400011F90123B371002C34D16B4699892B6886
:10415000C9BA4B4329891B4A1B145B1853806B4611
:10416000D9896B6849BA89B24B4369891B0C5B18C2
:104170001548191C1BB2834200DD011C0B0400D53D
:1041800000211388918001331380200005B0F0BD19
:104190000227220003AB3000009700F0F7F80E234F
:1041A0000400297C0122300000976B4400F0EEF8F7
:1041B0000443C3E71C00E8E7D441FF1FA061FF1FD1
:1041C00083050000B861FF1F0F27000073B5234E61
:1041D000300000F089F8224D07236A463000297C20
:1041E00000F002F904003000002C33D16B461B783C
:1041F0007F2B2FD800F0B6F86B46D878F023020456
:104200001B031A406B469B8816495BBA9BB21A4344
:104210002B68000953432A891B0C9B184B806B4663
:104220005A789B7812031B011A436B68024353436D
:104230006A891B0C9B180C481A1C1BB2834200DDB8
:10424000021C130400D500220B888A8001330B80E6
:10425000200076BD00F086F80124F9E7D441FF1F65
:10426000A061FF1FB861FF1F0F27000070B5114C40
:10427000237C002B0FD0382B0ED10F4D280000F0DF
:1042800033F8CC23AC222800217C9B0100F0F4F809
:10429000280000F067F870BD084BE2899A42FAD115
:1042A000054D280000F020F800222800217C00F0B5
:1042B000C5F8EDE7A061FF1FD441FF1F8305000093
:1042C00010B5084B1A7C002A09D05B69002B06D078
:1042D0009847041E01D0FEF793FE200010BD012474
:1042E000F9E7C046A061FF1F70B5C17905000C0059
:1042F000631E9C411A4BE402E41849000460C9B2F1
:10430000007906F0D5F8E979687949000131C9B238
:1043100006F0CEF8E8790930C0B207F049FB002377
:10432000E36661332360AA795B3B002A0ED02268E2
:104330009A43023B134323600A23E361073323625A
:1043400000232363A3630133E36370BD22689A43B0
:10435000022313432360462363610633A361EFE71F
:104360000050004070B5002504000368DD66C07988
:104370000930C0B207F0ACFB2900207906F034F810
:104380002900607906F030F870BD0000F8B51E0015
:1043900006AB1D78002304681700E366616007F030
:1043A000AFFA01238022E3662B0027615200013B14
:1043B00008D207F05DFB08200A4A1168002D03D1DE
:1043C0002800F8BD2261F2E7236F034203D023697E
:1043D000013D3370013613685B1A032BEED90125BA
:1043E000EEE7C0466008FF1F70B51C00002305689B
:1043F0001600EB66696007F083FA01238022EB6602
:1044000023005200013B08D207F032FB08200A4A81
:104410001168002C03D1200070BD2A61F2E72B6FD8
:10442000034203D02B69013C3370013613685B1AD9
:10443000032BEED90124EEE76008FF1F002370B5BF
:1044400004681500E366616007F05AFA0123E36629
:10445000256107F00DFB8020064A80001168636B20
:10446000034205D113685B1A032BF8D9012070BDF4
:104470000020FCE76008FF1F70B51D0000230468E2
:104480001600E366616007F03BFA0123E3662661EC
:104490000F33626B1A42FCD02B0A23611023626B2C
:1044A0001A42FCD0EDB2256107F0E2FA8020074AFB
:1044B00080001168636B034205D113685B1A032BFC
:1044C000F8D9012070BD0020FCE7C0466008FF1F3E
:1044D00070B51E00002305681400EB66696007F0E4
:1044E0000FFA0123A619EB660F33B4420ED107F081
:1044F000BFFA80200A4A800011686B6B03420CD11E
:1045000013685B1A032BF8D9012070BD217829614B
:10451000696B1942FCD00134E7E70020F5E7C0469B
:104520006008FF1F10B5084CE368002B08D18022FB
:10453000064B52021B689B186360054B1B68236087
:1045400007F0EEF8A06010BDE061FF1FC8F000406A
:10455000CCF0004070B5184A936A916A9942FBD139
:1045600016498A689A421FD39A1A8B60144B012607
:10457000186893B2D202D20E4343424300204C68E3
:104580001B0A1B1912029B180E4C0A684B60551C23
:10459000A3420CD8002801D04B600A600A4A13607D
:1045A00008680A4B186070BD581E821ADDE7084A79
:1045B00030009B182A00EAE700F00040E061FF1F8E
:1045C000140AFF1F40420F00C8F00040CCF000402A
:1045D000C0BDF0FF70B51F4C23793F2B01D93F239D
:1045E00023711D4B22791A701878C0B206F0F0FFC3
:1045F00018231A491A4A0B801A4913800B805380DA
:10460000A379194980200B800C21938001334B43FF
:10461000164D191C0001834200D9011C2980D1804C
:104620006379002B11D101336371237A012B01D8F7
:10463000022323726279237A0D4853430A21584397
:1046400006F0BEFF0B4D286070BDA02BEDD9A02356
:10465000EAE7C046D461FF1F480AFF1FEE41FF1F73
:10466000BC43FF1FEC41FF1FEA41FF1FE841FF1F52
:1046700071020000C461FF1FF8B514210020FEF78D
:10468000ADFE114C011E114D09D10C22104BC1CBB6
:10469000C1C4280007F04CFAFFF79CFFF8BD0C22BC
:1046A00020000C49FEF76EFE0C2802D0084B43CBCD
:1046B00043C40C2228000849FEF764FE0C28EBD006
:1046C0000C220021E5E7C046D461FF1FA061FF1F57
:1046D0001CBD0011FC0C0000F50C0000F0B51D4CD9
:1046E0008022A5440400882069465201400507F055
:1046F00007F8902212016A441300200032C832C326
:1047000016C816C38023144C144FA6689B0333436A
:10471000A3603B6007F084F98823A0685B05C0189C
:1047200007F0CEF80025882329008022A0685B05C9
:10473000C01840196944520007F0BAF980230135C6
:10474000FF355B019D42EED1A6603E60044B9D4467
:10475000F0BDC046FCEFFFFF2C43FF1F9808FF1F72
:1047600004100000F0B5040087B0002825D068468A
:1047700007F0B6F81B4C022806D106226946200035
:1047800007F026FA002816D06946002301250F26D7
:104790002F00E25C013310091030874038002F00F1
:1047A000324097403A0002434A610439062BEFD168
:1047B0006846FFF793FF07B0F0BD182269460A4824
:1047C00006F09EFF6A46A300D358013305D0182295
:1047D000FF21684607F0ACF9EAE70134062CF1D175
:1047E000E9E7C0466509FF1F00090011F0B5002583
:1047F00004000E0085B0AA4200D186E04B1C087868
:1048000001934B788978377909021943F3783F0689
:104810001B040B431F43039720706570252800D1AC
:1048200096E033D8112813D807F062F869002B01FD
:104830002B012B012B01AA00B800B1002B012B0189
:104840002B012B012B012B012B012B010501250134
:10485000232800D1DEE0DB2800D034E1042A00D890
:10486000ACE01025052A05D0551F2A003800711D1F
:1048700007F006F905223100200007F001F92A00AF
:104880003900601D07F0FCF805353EE0562859D088
:1048900010D8332800D19DE0552839D02628DAD108
:1048A0009F4B2900132218001D0007F041F9FEF765
:1048B000A7FB5CE0712800D177E0722800D180E08E
:1048C000602800D18BE0DC28C5D1022A00D875E031
:1048D0007378BFB26370B378A370032A05D0033A2C
:1048E000390092B2F01CFEF787FC10223900E01C60
:1048F000FEF748FDC51C002807DA60705CE00C225A
:104900002000884907F0BCF80C25280005B0F0BD50
:10491000013A854D0C2A13D8002A0AD028000199A3
:1049200007F0AEF8FFF756FE0C2228007F49FEF78D
:1049300063FC29000C22601C07F0A2F80D25E4E7B7
:104940000C22EBE7784D7A4B2A0043CB43C2E9E7D0
:10495000013A734D0C2A11D8002A08D00199280079
:1049600007F08EF80C2228007249FEF745FC29005A
:104970001322601C07F084F81425C6E70C22EDE72B
:1049800005226D49601C07F07BF80625BDE7122261
:104990006A49601C07F074F81325B6E708226849D5
:1049A000601C07F06DF80925AFE77178F02905D88C
:1049B000644B188801F09CFD0225A6E7FF23637075
:1049C000FAE7614B012A03D072789A706270F3E7BC
:1049D0009B78F4E72000FFF7E1FA050095E7013A3C
:1049E000594B5A4D072A10D8002A10D0012128000F
:1049F0005970019907F044F801F058F8290007228E
:104A0000601C07F03DF808257FE70722EEE700224B
:104A10005A70F3E7042A04D94D4D2F6006F080FE4A
:104A2000A860FFF797FD0422039003A9601C07F01C
:104A300027F8052569E7474D062A15D906222800DB
:104A4000019907F0C5F800280ED006220199280028
:104A500007F016F8062240492800FEF7CDFB012397
:104A6000394A91780B43937029000622601C07F0A5
:104A700007F8072549E7012AA0D07078FFF772FEF2
:104A80009AE7012800D0E6E6931E344F132B04D892
:104A90007378002B09D100F015F9314B39001D78DE
:104AA000601C6A1E06F0ECFF2FE7551E2A000199D4
:104AB000380006F0E5FF2B49AAB23800FEF79CFB50
:104AC00000F038F9E9E7DA281DD1042A00D875E7A3
:104AD000082A15D9B37972791B021343F2791204AB
:104AE0001A43337A1B0613433B603B6805223100AF
:104AF0002000039306F0C4FF0422601D03A950E7C1
:104B0000FE236370F1E7DE2800D057E7511E012A2B
:104B100001D10025F9E6019800F0AEFFF9E7C046A3
:104B2000A061FF1F28BD0011D461FF1FFC0C000015
:104B30001CBD0011F50C0000AC61FF1F8C61FF1F54
:104B40003043FF1FF041FF1FD061FF1F8D42FF1F49
:104B5000E061FF1F6509FF1FADAC0000D163FF1FBF
:104B6000CF63FF1FAEDE000070477047020010B534
:104B7000094B0A32094C92B2DA815A829881188222
:104B8000207802F01BFB0422054B012120781A70CB
:104B900006F02EFE10BDC046BA42FF1F1A64FF1F6A
:104BA0001964FF1F013870B5042809D806F0E8FF22
:104BB000030928081200234B0221187806F018FE7A
:104BC00070BD204B0821187806F0FAFF00221E4B1A
:104BD0001A72F5E7802200241B4B1A4D52001A81ED
:104BE00008211A682878DC7206F01AFE210028785D
:104BF00006F0AEFF012000F05FFE00F057FFDFE798
:104C0000104B0821187806F0DBFF1048FFF764F816
:104C10000F4B104A9B79002093800F4A138080220B
:104C2000094B5200D8721A8100F046FE00F03EFF98
:104C30000A4B9B78002BC3D0094A136006F070FF23
:104C4000BEE7C046F061FF1FC461FF1FF941FF1FAF
:104C5000D461FF1FBC43FF1FEA41FF1FD061FF1F4C
:104C600034F0004010B501290BD1012809D1054BC2
:104C70001B78002B05D02622034B04485A72FFF7FD
:104C800075FF10BDF263FF1FC461FF1FC409000060
:104C90000300F0B50A4D8E18B14202D152008018BF
:104CA000F0BD0C782F6824093C5D0F271C700C7830
:104CB00001313C402F683C5D5C700233ECE7C0463C
:104CC000E441FF1F0D22124B10B51A700C23114C3A
:104CD00011492370093A033B1048637006F0D0FE77
:104CE0002D2301220E490F48A371FFF7D1FF0122A6
:104CF0000D49FFF7CDFF01220C49FFF7C9FF030063
:104D000000200B4902001870FEF776FA10BDC0466D
:104D1000EE63FF1FCF63FF1FDBBC0011D163FF1FDA
:104D20006709FF1FD663FF1F6609FF1F6509FF1F85
:104D3000AEDE000070B5124C142220001149FEF7BF
:104D400021FB431E104D132B17D8AB78002B14D02A
:104D5000431C2B7009236B70002300190370287803
:104D600029000130C0B206F033FD29782200013954
:104D7000C9B2002005F0BEFD70BDFFF7A3FFEEE74E
:104D8000D163FF1FAEDE0000CF63FF1F10B5114BD4
:104D90001A781870002A0ED000280BD10E4B1A7802
:104DA000062A07D85423D340DB0703D50B4B1878CA
:104DB00002F004FA10BD0028FCD0074B1B78012B31
:104DC00002D0033B022BF5D8044B0121187806F0E2
:104DD0000FFDEFE7F263FF1F1964FF1F1A64FF1F47
:104DE00070B54A4E4A4A4B493070012005F00EFC1E
:104DF00000F0C0FEFEF704F906F03AFD0322464932
:104E00004648FFF745FF2D24030004221C70444947
:104E10000130FFF73DFF30230470424D424C437098
:104E200083702E3B062220004049EB87FEF7AAFA4A
:104E3000062813D0200006F053FD022809D00321D4
:104E4000200006F0ADFD8D23E3706E3B2371193316
:104E50006371062220003549FEF7CEF9344B1B68FA
:104E6000FC335C64FFF766FF0020FFF78FFF314CD7
:104E7000314A0121314B1278207802F061F9304A31
:104E8000304B12780021207802F05AF901222E4B83
:104E90001A702E4BDB78552B31D12D4B3B325A7289
:104EA0002C4B2D4AAB81EA812B826A8220213078FB
:104EB00006F02EFE0120404205F068FD0120404230
:104EC00005F004FEFFF71AF9FEF7CEFE00F0B2FC83
:104ED00001204042FEF7A4FF012006F031FEF02041
:104EE00001F0EAFA0121307806F082FC307802F015
:104EF000C1FA1A4806F06CFDFEF772FD70BD64221F
:104F0000174B5B7953431A000A32CBE7F061FF1F5E
:104F1000694B0011654C00113043FF1F8C61FF1F6E
:104F2000AC61FF1FBA42FF1F6509FF1FADAC000057
:104F30004464FF1F1A64FF1F1842FF1FF941FF1F3F
:104F4000EE63FF1FCF63FF1FC063FF1FD061FF1F12
:104F5000C461FF1FC4090000CE090000F261FF1FF9
:104F6000D461FF1FF8B50A0020230D001A40194232
:104F700063D05E4B1B78002B5CD0FFF7EBFA5C4BE9
:104F80005C4C5D4E99686268737A8A1ADB039A42B8
:104F900002D36160FEF724FD327A217A531EDBB220
:104FA000994205D1FFF762F9002000F0B5FD15E048
:104FB0009142F9D300272772FFF782F9A37ABB4207
:104FC00002D0A772FEF792FD012000F0A5FD4B4F25
:104FD0003800FEF781FE390006F07AFC637A002B78
:104FE00025D0013BDBB26372002B20D1444BDB7830
:104FF000552B01D106F094FDE37A002B12D000234B
:10500000A27AE3729A4202D0A372FEF76FFD3D4A84
:105010003A4F1388380001331380FEF75DFE3900E4
:1050200006F056FC642370795843FFF79FFD237AFE
:105030000133237220206840F8BD0BB2002B0ADA3E
:10504000314B187806F0E4FC002801D006F0F8FA9D
:1050500080200002EFE70224214206D0254B0120E8
:105060001A72FFF793FE2000E5E70B071ED5FFF746
:1050700071FA1F4B1F49204C98684A68637A821A5C
:10508000DB039A4202D34860FEF7AAFCFFF718F947
:10509000FFF7ECF8012000F03FFD00F0E5FB23688E
:1050A000DB0701D5FEF7B4FF0820C4E7CB0609D51E
:1050B000FEF71CFD0D4B1B78002B01D1FEF7E8FD20
:1050C0001020B8E70124214207D0104800F06CF806
:1050D00006F036FC00F006FDC5E704240800204079
:1050E0002142A9D0FEF7B8FEBDE7C046F263FF1F1C
:1050F000E061FF1FC461FF1FD461FF1FF941FF1F63
:10510000D061FF1FB861FF1FF061FF1FDC41FF1F6F
:10511000F0B51B4B1B4F1B883A8804001A4E1B4DE1
:1051200085B09A420DD832889A420AD3184B1A8811
:105130002B889A4205D1174A174B12881B889A422E
:105140001BD0052001F00EFA3B8802AA1380338899
:10515000019053802B88114D93800F4B02A91B881F
:10516000D3800F4B2A78188802F02AFF0D4B0821B4
:105170002878019A1C7006F0ABFA05B0F0BDC04665
:10518000BE63FF1FEE41FF1FEC41FF1FEA41FF1FFF
:10519000BC63FF1FBA63FF1FE841FF1F1A64FF1FB4
:1051A000F041FF1FB863FF1F13B50C4B1C78002C98
:1051B00011D1002801D00A4B18600A4A0A4B117815
:1051C0000A4A10780A4A01920A4A0092002205F01F
:1051D00089FA200016BD1124FBE7C0461964FF1FA1
:1051E000B463FF1F1864FF1F0864FF1F1A64FF1FCA
:1051F000F463FF1FF863FF1F10B5064B12201B78E6
:10520000052B06D1044B13221988044B187801F0A2
:1052100085FB10BD1964FF1FF041FF1F1A64FF1FBB
:1052200010B500240122114B52421870104B1C7013
:10523000104B1A8002F01EF904220F4B21001A7045
:105240000E480C3206F00CFA102221000C4806F031
:1052500007FA07220B4B1C600B4B1C700B4B1C708E
:105260000B4B1A700B4B1C7010BDC0461A64FF1F0D
:105270001964FF1FF041FF1F1864FF1F0864FF1F20
:10528000F863FF1FF463FF1FCE63FF1FCD63FF1F93
:10529000F241FF1FCC63FF1FF8B5174C06002578BD
:1052A00006A814240078052D23D1B41F134FA5B2EE
:1052B0001824BD421DD88D1FADB2BD4219D8FA25A4
:1052C0006D00AA4215D21D000D4F0A3DADB2BD4280
:1052D0000FD80C4C26800C4C21800C4900240A80ED
:1052E0000B4A1380FFF714FF0A4B0421187806F0CD
:1052F00067FC2000F8BDC0461964FF1F790C000050
:10530000750C0000EE41FF1FEC41FF1FEA41FF1F3B
:10531000E841FF1F1A64FF1FF0B50BB20D0089B002
:10532000002B00DB70E1A44E307806F071FB041E08
:1053300050D00378A22B00D122E1D02B1AD0912B90
:1053400045D143780E2B42D19C4B82889A423ED164
:105350009B4A83681278052A39D1032018567F2882
:1053600035D0984B1B68002B31D05B68002B2ED0BA
:1053700098472CE08078072829D806F001FC0428FB
:10538000183F3F74A8D86378002B0CD101218C4BB7
:1053900019708D4B1A78002A5BD08C4B307801F055
:1053A000CFFE002855D00722854B1A7051E0617856
:1053B0000029F8D1E378002B11D0854A854B12786B
:1053C000307801F0BDFE60706378002BEBD12000D7
:1053D00006F036F980200002684009B0F0BD784B35
:1053E0001B78022BF3D00121307806F009FB00284E
:1053F000EAD10121307806F0FBF9E5E76378002B6C
:10540000D1D16F4F032807D13B78052B02D101334F
:105410003B701EE00223FBE76F4B1A886F4B029331
:10542000002A0BD01B78002B03D00121307806F026
:105430004FF93B78062B04D1013BE9E7029B1A7038
:10544000F7E7042B41D10121029B3078197006F057
:10545000CFF95C4B1B68002BB9D01B68002BB6D072
:10546000574A107884E76378554F002B27D10622DE
:10547000211D5B4806F004FB62895A4B5A491A8089
:10548000A2895A4B1A80E3890B800521397058494B
:105490000A80584A1380228A574B1A80574B1B7830
:1054A000012B09D11F2001F05DF8FA22920042433E
:1054B0000421307806F00CF90022484B75E7312BB7
:1054C00000D070E70022454B1A700323A0E70622A4
:1054D0000021434806F0C4F80023454A0421138004
:1054E000444A30781380444A138006F069FB08214F
:1054F000307806F065FBA379083B5A425341304AA5
:1055000003331370304B1B78002B06D0334B3078AD
:105510001A78002A06D001F051FE0122314B524286
:105520001A8096E70121197006F062F9F5E7082163
:10553000307806F045FB6378002B00D047E72C4B12
:105540002D4F0293E388029A04211380294B30786F
:1055500003932389039A138063893B8006F050FAF2
:10556000002800D033E7264B1B68002B00D12EE724
:10557000039902983A88098800881B68984726E7AB
:105580004379132B00D022E70389012B0AD11D4B4D
:105590001B78022B06D10821307806F011FBFFF7AB
:1055A0002BFE14E7052000F0DDFF08210200307813
:1055B00006F08EF80BE7C0461A64FF1F05140000C2
:1055C0001964FF1FB463FF1F1842FF1FF941FF1F3B
:1055D000EE63FF1FCF63FF1FF063FF1FF263FF1F28
:1055E000C163FF1FF041FF1FC863FF1FCA63FF1F96
:1055F000BE63FF1FBC63FF1FBA63FF1FC063FF1FB3
:10560000B063FF1FB863FF1F8020C001014200D0BC
:10561000E2E6CB0731D5324B1B78002B1DD0314E43
:1056200005AC3378052B1AD1023B23702E4B210099
:105630001B7823722D4B1B7863722D4B187801F069
:1056400023FD002809D007202A4B30701B68002B4F
:1056500003D01B68002B00D098470120BCE60E2029
:10566000254B06221B7825492370254B1B78637038
:1056700002ABC01806F004FAD8E70223080018406D
:10568000194209D0174B1B78052B03D11D4B1888E5
:1056900006F04EF802209FE60424214203D0FFF7D3
:1056A00037FD200098E6082308001840194200D171
:1056B00093E6154B1C78012C03D0022C0DD008204A
:1056C0008AE6124B124A134913481B88128809882C
:1056D00000880094FFF7E0FDF1E7FFF78DFDEEE7AE
:1056E000F263FF1F1964FF1FF241FF1FCC63FF1F0E
:1056F0001A64FF1FB463FF1FCE63FF1FF341FF1F38
:10570000CD63FF1FF041FF1FB863FF1FE841FF1F7C
:10571000EA41FF1FEC41FF1FEE41FF1F10B502A839
:1057200004880B20002C10D14968087849780902B8
:1057300001430C48814209D1022119800A4B598842
:105740001170DB7800205BB2537010BD074C0A204B
:10575000A142FAD102211980034B998811705B791B
:10576000F0E7C0466E2A0000B861FF1F6F2A0000F4
:10577000F7B5150008AA16884A680F4F14785278B2
:10578000120222430A24BA4214D10122DBB201924E
:1057900000962A0005F0ACFE041E0BD1074B1B68D7
:1057A000002B07D068782A7800021043424250410B
:1057B000013098472000FEBD022900002C64FF1F25
:1057C00030B5012503790400BFB02B4225D0144920
:1057D000408805F0F9F928420CD0124B01A95B8DE5
:1057E00000220B8002234B800F4B5B888B806088EC
:1057F00002F0DCFA0D49608805F0E6F9C0070CD527
:105800000B4B01A91B8800220B8002234B80064B07
:105810009B888B80608802F0C9FA3FB030BDC046DB
:105820002464FF1F1C42FF1FB861FF1F1C64FF1F81
:105830007642FF1F10B5074C0749200005F07AF9A2
:105840002000064905F076F90721054A054805F0CC
:1058500033F910BDFFFF00002464FF1F1C64FF1F0D
:1058600048BD00111C42FF1F10B5024803F020F98B
:1058700010BDC046C15700110221430888400B40AB
:105880000A31084003430E20024AD17881430B437A
:10589000D37070478D42FF1F064A1379410705D523
:1058A00080210B4380011371907170477F210B4061
:1058B000F8E7C0468D42FF1F054A5378002803D001
:1058C00080210B43537070477F210B40FAE7C0469D
:1058D0008D42FF1F0F21114BDA780A40DA705028F1
:1058E00010D901310A43DA702022D9780A43DA70DC
:1058F0004022D9780A43DA708022D97852420A438A
:10590000DA7005E03C28EFD82828F1D81428F3D81D
:105910000122D9780A43DA707047C0468D42FF1FD2
:10592000F8B57F23324D04006E789E43314B984288
:1059300005DD76232B70363B33436B70F8BD2E4B61
:10594000984203DA58232B701433F5E783B21A0018
:1059500000215F32294892B2294F297082422DD905
:10596000A9708C4203DA5B421CB220232B700534F1
:1059700020B20A2105F024FE04B2FA239B009C42C7
:1059800033DB80232A785B4213432B706421200091
:1059900005F016FE0A2100B206F0A2F809B22A7834
:1059A0007B5C13432B700A21200005F009FE0A21BD
:1059B00000B206F095F809B27B5C0AE08022AA707A
:1059C000002CDADA5B421CB220232B705F23092CF7
:1059D000E9DC1E430A2120006E7006F081F809B24E
:1059E000AA787B5C1343AB70A8E7632CCEDCEDE7B1
:1059F0008D42FF1F1B4E00001DFCFFFF2A08000008
:105A000072BD00117F23F7B5194FCD013E79040017
:105A10009E433E71EDB2632806DD093B33433B7183
:105A200040231D437D71F7BD0300093304DA582379
:105A300033433B716C23F4E70E4B019300280BDAE0
:105A40000423444224B23B710A21200006F048F8A6
:105A5000019B09B25B5CE4E70928F5DD0A2105F04A
:105A6000AFFD019B00B21B5C1E433E71ECE7C046DC
:105A70008D42FF1F72BD0011F8B50A4F05003B783B
:105A80000E00002B0CD0084C2000FEF72DFC33003C
:105A90002A0020003978FEF71BFD2000FEF762FC8B
:105AA000F8BDC0463864FF1F9442FF1F70B50A4E10
:105AB0000A4D07223100280006F08AF8002809D094
:105AC000074C31000722280005F0DAFF08212000EA
:105AD000FFF7D2FF70BDC0468D42FF1F3164FF1F2C
:105AE0003064FF1F7F2210B50A4B59789143033A67
:105AF0001A70103A0A435A7078220E219A70DA7896
:105B00008A43DA7006221A7130325A71FFF7CEFFDB
:105B100010BDC0468D42FF1F10B5002824D0134C85
:105B20000A210223E05E05F04BFD00B2FFF7F8FE0C
:105B30000423E05E642105F043FD012100B2FFF77C
:105B400061FF207AFFF7C6FE0320FFF795FE0020D5
:105B5000FFF7A2FE064B1878053843425841C0B201
:105B6000FFF7AAFEFFF7A2FF10BDC046B861FF1FF6
:105B70001964FF1F70B50024094D2800AC71FEF7B1
:105B8000B3FB10233E212800064AFEF7A1FCA042E9
:105B900000D13E34044B28001C70FEF7E3FB70BDBF
:105BA0009442FF1F62BD00113864FF1F0200F0B570
:105BB00001270A480A4E51188B1A002B00DCF0BD51
:105BC000082415784308684038404000805B013C59
:105BD00058406D08002CF5D10132EDE7FFFF0000C1
:105BE00082BD0011F0B500250F269D4200DBF0BDFF
:105BF0004C5D070944403440A400A058013578406A
:105C0000F3E70000F0B589B06A460D000B000F27DE
:105C1000110010351C780133260024093E4016700F
:105C200054700232AB42F5D12023024AFFF7DAFF6B
:105C300009B0F0BD88BD0011F0B54E780B7889B081
:105C400036020C00170001901E43012A61D9954BC2
:105C50009E4200D877E001339E421CD1062A17D11C
:105C6000CA788B7812021A430B791B0413434A79C2
:105C700012061A438C4B5A6100221A705A808B4AC2
:105C80005A608B4A9A608B4ADA60002009B0F0BDF6
:105C900088225205EEE7884B9E423CD182498B78A0
:105CA000002B00D0F6E00C2A31D10F22A3789343C9
:105CB000E278120213432279120413436279120626
:105CC00013434B60E279A07912020243207A000468
:105CD0001043627A12060243CA60E27AA07A120284
:105CE000024376484A81834208D804236E4914222D
:105CF00001980B7005F0C4FE1420C7E71201D218FA
:105D000089235B059A42F0D801238B70BDE7022AF4
:105D1000FAD00523EAE76A4A01239642E6D1FFF763
:105D20006BFA052F0CD9E378A2781B021343227972
:105D300012041A4363791B061343624A03931360E8
:105D400005F0EEFEA1E7584D2B78002B9DD1AB78E6
:105D5000002B00D1A0E02B8901339BB20093B3420A
:105D600000D091E0132AD4D9CF7C8B7C3F02122142
:105D700020001F43FFF71AFF874200D08EE0002E5D
:105D80003DD1E378A2781B0213432279E96812041B
:105D90001A4363791B06134303930A228B4212D1E1
:105DA000FF23A370E370237163716B89002B09D10A
:105DB000E37B227C1B0212041343A27B13431B09C7
:105DC00001336B8100226B89002B8ED0002A67D1B2
:105DD000686837013818000B6B690003039098421C
:105DE00005D9686105F06CFDEB780133EB706868EC
:105DF0001022A11C381805F05BFE2E8145E76F8943
:105E0000009A7B1E9BB293423AD1E278A3781202A9
:105E10001A43237905A81B04134362796C681206A0
:105E20001A43EB6800920392211D0C22049305F0A3
:105E300027FE0120260004A940421036FFF7E2FEAB
:105E4000013F012F17D1009A0B232861824200D015
:105E50004CE704221C49200005F02AFE042203A975
:105E6000686805F04DFCE968039AFF23914200D170
:105E70003CE7F73B3AE73100FFF7C4FE1036DFE7B7
:105E80000923B742A4D831E7009BB34200D9FCE60E
:105E900007232BE7022329E7032327E7062325E728
:105EA0000A2323E7FFFE00009C42FF1F00000111B0
:105EB000FFFF00005048593601FF0000FFFF0011AE
:105EC00002FF000034F00040A842FF1F10B5034C51
:105ED0000B000122210000F06BFA10BD8D60001153
:105EE0000B8870B506000D000224162B11D92B006B
:105EF0000322094900F05CFA041E0AD1074B2A88E4
:105F00001B88191C934200D9111C300089B200F083
:105F1000EFFA200070BDC046B96000114A64FF1F4F
:105F200010B54A780400013A0B000220012A07D874
:105F30000A78002A04D005222000024900F038FA2D
:105F400010BDC046E76000110A7810B50B000400D0
:105F50000220002A04D007222000024900F028FA7B
:105F600010BDC046936100110A7810B50B00040003
:105F70000220002A04D009222000024900F018FA69
:105F800010BDC046F961001110B5034C0B000B2287
:105F9000210000F00DFA10BD2962001110B5034C6C
:105FA0000B000D22210000F003FA10BD9B620011CE
:105FB00010B5034C0B000F22210000F0F9F910BDC1
:105FC000F56200110A7810B50B0004000220002AC7
:105FD00004D011222000024900F0EAF910BDC046A9
:105FE00005630011002310B51322190000F0E0F939
:105FF00010BD000010B5034C0B001722210000F06B
:10600000D7F910BD57630011002310B519221900EC
:1060100000F0CEF910BD000010B5034C0B001B22A0
:10602000210000F0C5F910BD91630011F7B5848916
:106030000D0006000121002C22D000238268D356D7
:106040001778002B1EDA0C2C1AD90C3CA4B21319A9
:1060500040880093230002F086FE431E98410130E1
:106060007B06DB0F6B703F23013C1F40A4B22870FE
:10607000AF70AC80002C07D0B3680133AB60002157
:106080000800FEBD0020EBE7AC60F8E70B7803707A
:106090004B8843704B881B0A83700B79C3700420B4
:1060A00070470420022B06D10020537811781B0280
:1060B000009A0B43138070470B8803700B881B0AF0
:1060C0004370022070470420009983420AD153781C
:1060D00010781B0203430B80D37890781B02034394
:1060E00000204B807047F8B50D004B78012400214B
:1060F000461C03702B788B4201D82000F8BD6B78CA
:10610000B01C4F1C012B10D1890069184B8802224A
:1061100033704B88B9001B0A7370691805F070FA68
:1061200004360434A4B2F9B2E4E7122359436B18DD
:106130005A88043132705B8810221B0A7370691808
:1061400005F05EFA12361234ECE770B5049D1400C7
:106150001E00052B01D8042070BD637812781B0245
:1061600013432B80E378A2781B02134302226B8037
:106170002A71211D681D063E05F042FAB2B22A813D
:10618000E92AE8D82800A11D0A3005F039FA0020D4
:10619000E2E7002310B50A789A4201D8900010BDBA
:1061A0009A008A185488013304705488DBB2240A98
:1061B0004470948884709288120AC2700430EAE7AE
:1061C00010B51100029C062B04D004201022142BC1
:1061D00001D010BD022222714B7808781B020343C4
:1061E0002380CB7888781B02034363800431601DD1
:1061F00005F006FA0020ECE710B50C788B78043136
:106200005C43E4B203702200013005F0F9F9601C30
:1062100010BD0420022B06D10020537811781B02F8
:10622000009A0B431380704710B50C000A880231A6
:1062300005F0E6F9208810BD70B504000D00049843
:106240001100012B01D8042070BD1678527812027B
:10625000324302800200F13255701470E125002CA7
:1062600000D10C35023B9AB24280AA42EBD80231EF
:10627000043005F0C5F90020E6E7042000998342C8
:106280000AD1537810781B0203430B80D37890789F
:106290001B02034300204B80704710B50C000A8896
:1062A000023105F0ADF9208810BD000070B5012164
:1062B0001E000420049C0E400B4218D1CB40DDB2DE
:1062C0008D4214D90A49DBB2098899420FD32300C1
:1062D000EE331D703300580011184978165C09021E
:1062E000314301332152D9B28D42F4D8002070BD20
:1062F000B442FF1F10B50C000A88023105F080F986
:10630000208810BD10B50C788B7804315C43E4B262
:1063100003702200013005F073F9601C10BD10B548
:1063200011000298032B01D8042010BD1478527874
:10633000043B120222430280CA788C781202224364
:1063400042809AB28280EB2AEED80431063005F002
:1063500057F90020E9E710B50C000B8803700B8893
:106360001B0A43704B8883704B881B0AC3708A8852
:106370000430063105F044F9A088043080B210BD25
:106380000420012B03D100201378009A137070476A
:1063900010B50C000B8803700B881B0A43704A88E9
:1063A0000230043105F02CF96088023080B210BD53
:1063B000F0B589B003931E4B029242000700D05AF9
:1063C000019102F020F81325061E2DD0029B012416
:1063D0000370019B002B04D0001903999847001902
:1063E00084B26B461B7A5BB2002B0FDA10213800A7
:1063F00002F01CFB1925002813D130003219E1B23C
:1064000002F066FC051E0CD10C34A4B2042304AACD
:10641000380005A993800696948101F0AFFD051E12
:1064200002D0300005F0BCF9280009B0F0BDC0462C
:106430004864FF1F70B505000C0000280CD0002038
:10644000814209D010222000044905F0D9F801202A
:106450002B7823736B78637370BDC046C8BD001181
:10646000F0B506000D0017001C0085B002291BD0F6
:106470000020102907D1022B07D0102B03D115E0E3
:106480000020102C08D005B0F0BD69463800FFF799
:10649000D1FF2A0069460BE069463000FFF7CAFFCA
:1064A00022006946380004E0022BE9D12A003900B5
:1064B000300005F025FBE6E7031CF02800D9F023A7
:1064C000032008499AB2013A0B80D31703400649CA
:1064D0009B189B100B80D30F04499B185B100B80FB
:1064E0007047C046B842FF1FB642FF1FB442FF1FAD
:1064F000034B1B888B4202D3024B4000C1527047B2
:10650000B842FF1F4864FF1F014B4000185A7047F4
:106510004864FF1F1722014B1A8070474864FF1F11
:1065200070B505000E2005F03BFB041E13D0D023F0
:10653000037000230622837007494570033005F07D
:106540005FF8064B2100DA8A62811B7E2373044BBD
:10655000187805F05DFB70BD6464FF1F5464FF1F75
:106560000843FF1F262803D8024B4000C05A70473B
:106570000148FCE7BA42FF1FFFFF000070B50600AC
:106580000C00094D1C220021280005F069F8074B7A
:106590001E70074B1C7005F063FA0123002801D020
:1065A000002312202B7070BD5464FF1F0843FF1F8F
:1065B0007564FF1F70B505000D4C0800E260A16016
:1065C00010220021656005F08BF8012803D110210D
:1065D000A06802F058FD10220021280005F080F884
:1065E000012803D11021606802F04DFD70BDC04646
:1065F0005464FF1F70B5041E05D1002903D0062284
:106600000D4804F0FDFF0D4B1D78012D11D1002C1C
:1066100005D102221A7004F0EBFF280070BD0022A1
:106620001A70074B1B78FF2BF7D02000FFF778FF7D
:10663000F3E70025F1E7C0466464FF1F5464FF1FC1
:106640000843FF1F030010B5002801D1002010BD32
:1066500000780B4A002803D15988D1821B79137620
:106660001378022BF2D10023984200D10333137028
:10667000044B1B78FF2B01D0FFF752FF0120E6E708
:106680005464FF1F0843FF1F002911D000280CD0BD
:106690004B79012803D140225242134303E03F22A9
:1066A0001340032802D001204B7170474022F4E7C9
:1066B0000800FAE770B5094D0100287800280BD0D2
:1066C000074C0622200004F09BFF21002878FFF7EA
:1066D000DBFF200005F0ECF870BDC0467464FF1FBE
:1066E0004E64FF1F00290AD0012808D13F224B79B0
:1066F0009343C02B03D0403B5A425341981C7047F0
:1067000070B5174D06002B78FF2B15D00A2005F029
:1067100047FA041E10D0D0230370C83B8370114B7E
:1067200011491B784670C3700622043004F068FFDC
:106730002100287805F06CFA0C4B1B78012B0DD149
:106740000B4B1B68002B03D09B68002B00D0984795
:10675000084B04211878084A05F062F870BDC0465D
:106760000843FF1F7464FF1F4E64FF1F7064FF1F08
:106770009C64FF1FA064FF1F60EA0000014B986843
:106780007047C0465464FF1F014BDB6818687047B0
:106790005464FF1F074B10B5DA68136801331360A8
:1067A000054B1878FF2803D08021C90105F020F897
:1067B00010BDC0465464FF1F0843FF1FF7B50E000D
:1067C00002F0C8F8051E1CD00E4B06621F78002F81
:1067D00000D10778AB791020019305F0E1F9041E90
:1067E0000FD0D0230380C73B8370019BE91DC3708A
:1067F0000622043004F004FF21003800E66005F0B2
:1068000007FAF7BD0643FF1F014B18787047C046D3
:106810007464FF1F054B002805D1054B1A78054B02
:10682000002A00D1014B18007047C0466464FF1F66
:106830007464FF1F4E64FF1F014B58687047C046C9
:106840005464FF1F024B1868431E9841C0B2704742
:106850007864FF1F421E03000120152A03D9FF3B65
:106860005A425341D8B27047F0B51C0000230E00C5
:1068700085B0039002920B70029A934201D30020DC
:1068800019E0E55C5A1CD2B2002DF8D002985119DB
:106890008142F4DC0233DFB2A35C18000193FFF7FE
:1068A000D9FF002807D0013D019A0399EBB233705C
:1068B0008A4202D1E01905B0F0BDDB19DBB2DBE79B
:1068C00010B50C0002F09EF803001220002B03D03C
:1068D0002100588804F094FF10BD000070B50E4DE3
:1068E00084006359002B15D0186A002801D004F0E9
:1068F0009FFE2B59586A002801D004F099FE2B59AD
:10690000986A002801D004F093FE285904F090FE04
:1069100000232B5170BDC0468464FF1F1C4B70B513
:1069200004000E00150099420AD11A4B1B68002B77
:1069300001D1122070BD1B68002BFAD09847F9E7EF
:10694000154B994215D1134B1B68002B0AD01B68BD
:10695000002B07D09847002804D1104B1C70104B17
:106960001D70E7E729002000FFF7AAFF0028E1D10A
:10697000F3E7080001F0EEFF0028DAD003780320E7
:10698000A342D7D12900300004F03AFFD2E7C04635
:10699000FEFF00008064FF1FFFFF00007D64FF1FFB
:1069A0007C64FF1FF7B50400808801F0D3FF002549
:1069B000A84203D00578A08802F008F81C4E33786E
:1069C000002B1FD0AB421DD11A4B28001978FFF7BE
:1069D00077FF002818D000233370A3790820A77808
:1069E000A688019305F0DCF8011E0DD0D0230370BA
:1069F000CA3B8370019B477086808371280005F035
:106A000007F901E0002DE8D1A0880B4B8200D35894
:106A1000002B01D0FFF762FF1721A088FFF768FD68
:106A2000A08801F027FDA08801F0FEFDF7BDC0465B
:106A30007D64FF1F7C64FF1F8464FF1FF0B587B077
:106A40001D000CAB1B88070001930DAB1B881420A5
:106A500002930EAB1B88160003930FAB1B880091AB
:106A6000049310AB1B88059305F09AF8041E1AD006
:106A7000D0230370CB3B47708370C6700622290079
:106A80000430002D11D004F0BBFD019B2100638177
:106A9000029B0098A381039BE381049B2382059BB7
:106AA000A37405F0B5F807B0F0BD04F0D9FDECE72C
:106AB000F7B5009308AB1B8807000C200D001600EB
:106AC000019305F06DF8041E13D0280001F042FF79
:106AD00000280FD00078D0232370C93BA370009BFF
:106AE00021002381019B6770A580E680638105F00A
:106AF0008FF8F7BD014B1878EDE7C0460843FF1F3C
:106B000013B5040064890389C2888188C078009421
:106B1000FFF7CEFF13BD000010B5044C206800281D
:106B200003D004F085FD0023236010BD8864FF1F9F
:106B3000A122F0B5818892004A43384B384F1B6838
:106B400004009B189D2292009B18827989B01A60DC
:106B50003B68002B5FD01D78324B1B68002B04D0A4
:106B60005B68002B01D000209847260008363100D2
:106B7000E079FFF7B7FD237DE0710200E078049330
:106B8000638A29000393238A0293E3890193A388EC
:106B900000933300FFF752FFE378002B0BD1E2891B
:106BA000A379A18802920196E2792800009201223D
:106BB00001F0DAFEE0703B68002B20D0FFF7ACFF5D
:106BC000194D287800281AD0184B1978FFF778FE4D
:106BD000002814D02B78E67808200793A78804F0C3
:106BE000DFFF011E09D0D0230370CA3B46708370BB
:106BF00087808671079805F00BF800232B7017210A
:106C0000A088FFF775FCA08801F034FCA08801F093
:106C10000BFD09B0F0BD064B9DE7C0463409FF1FD0
:106C20008864FF1F9C64FF1F7D64FF1F7C64FF1F3F
:106C30000843FF1FF8B5070008000E0001F08AFEA8
:106C4000041E18D02620FFF78DFC051E00D12578E4
:106C5000062004F0A5FF041E0DD00021062204F03A
:106C6000FFFCD0232370C23B21006770A370A68075
:106C7000E8B204F0CDFFF8BDF0B585B001930AABE2
:106C80001B78070002930BAB1B7808000D000092E5
:106C9000039301F05FFE061E22D0102004F080FF57
:106CA000041E1DD01022002104F0DAFC2620FFF77C
:106CB00059FC002800D13078D0232370C13BA37049
:106CC000009B21002372019B67706372029BA58069
:106CD000A372039BC0B2E3720C9BE36004F098FFC5
:106CE00005B0F0BDF7B50D00019001F033FE071EB1
:106CF00020D00E2004F054FF041E1BD02620FFF7E6
:106D000031FC061E00D13E78D0232380C53B0622ED
:106D1000A370F91DE01C04F073FC019B2A00638141
:106D20000123DD401A401D40210022736573F0B23B
:106D300004F06EFFF7BD0000F0B585B002901000C2
:106D40000D0017000A9E039301F004FE041E31D0CB
:106D5000029B002B2ED1039B02795B0724D51223C3
:106D600013430422002E08D10B99002905D10C9958
:106D7000002902D10D9900291AD01A430D9B2271C6
:106D8000002B00D0C9E0002E00D1CFE0002D00D0B4
:106D9000CCE0606A002801D004F04AFC1C213000DD
:106DA00004F0D6FC606205E002239A430E33D7E775
:106DB00093432371654BBA00D458002C00D1AAE04C
:106DC000002E10D0236A002B03D11C2004F070FC8D
:106DD00020625E4BBA00D358186A002803D01C22E8
:106DE000310004F00DFC0C9B002B12D0574CBB0063
:106DF0001D596B6A002B03D1162004F059FC686200
:106E0000BB00E358586A002803D016220C9904F0FE
:106E1000F7FB0D9B002B11D04C4DBC006659B36A9B
:106E2000002B03D1142004F043FCB0622B59986A64
:106E3000002803D014220D9904F0E2FB380001F081
:106E400089FD051E67D0414BBA00D358002B62D094
:106E50001A6A3420002A00D11C389A6A002A01D00C
:106E6000143080B20B9A002A01D01C3080B25B6AC9
:106E7000002B01D0163080B204F092FE041E4AD0DE
:106E80001822002104F0ECFB2620FFF76BFB019099
:106E9000002801D12B780193D0232370029B20007E
:106EA00063700A23294EA370039BBD00A371AB59E5
:106EB000A780196A1830002905D01C22A06004F0B0
:106EC0009FFB200034307359996A002907D00300D2
:106ED00014221433E060029304F092FB02980B9B9F
:106EE000002B08D003001C221C330B992061029355
:106EF00004F086FB02987359596A002903D01622C0
:106F0000606104F07DFB6B462100187904F080FE7F
:106F10003800FFF7E3FC05B0F0BD10220D9B0D9982
:106F20001B69A018236204F06BFB2CE70B9B002B62
:106F300000D13FE7012D00D03CE7606A002801D076
:106F400004F076FB1C210B982AE7C0468464FF1FDF
:106F500010B5044C2068002803D004F069FB00231E
:106F6000236010BD7864FF1F0B4B07B51A68002A19
:106F700001D100200EBD6946531C01201278073153
:106F8000FFF772FC0028F4D00278012310001840AB
:106F90001A42EED0EEE7C0469464FF1FF0B51F4FD3
:106FA00001203B6887B0002B25D09B78059300F02B
:106FB000B3FB002821D00A20FFF7D4FA04000B20ED
:106FC000FFF7D0FA164B05001E78731E9E413B68F2
:106FD000F6B2191DD878FFF757FB3B682900DA7A1B
:106FE000043303929A7901930292009033002000B7
:106FF000059A04F04DFB07B0F0BDFFF7B5FF002880
:1070000005D00620FFF7AEFA04000720D8E70820D5
:10701000FFF7A8FA04000920D2E7C0467864FF1FF2
:107020007464FF1F70B50A4E040033780D00FF2B07
:107030000DD0042004F0B4FD011E08D0D02303704D
:10704000CE3B45708370C470307804F0E1FD70BDB4
:107050001843FF1F70B5040006200D0004F0A0FDCA
:10706000011E0AD0D0230370CD3B8370054B4470C2
:107070001B688580187804F0CBFD002C01D0FFF749
:1070800067FF70BD7864FF1FF8B5264F06003B68A8
:107090000D001124002B05D10522234B1B78134230
:1070A00002D112242000F8BD204A10241268002AC0
:1070B000F8D01278002AF5D0DB0719D52B789A1E64
:1070C000012A1AD80C2004F0F3FA1324386000289F
:1070D000E8D000230A22437029000670023004F031
:1070E0008FFAFFF75BFF041E0AD0FFF731FFD9E7E5
:1070F00000F012FB0028E1D1E4E7002BE2D0D0E75A
:107100000B4B1B78032BCDD11D20FFF72BFA094B1E
:1071100018800028C6D0084B04211878074A04F0CC
:107120007FFBBFE77864FF1F7564FF1F9464FF1F38
:107130007464FF1F7264FF1FA064FF1F60EA0000F9
:10714000F7B50193194B14001A78052306000F00B8
:1071500012201A4221D0012920D1154B1D68002D83
:107160001BD002201F2C18D8002C02D0019B002B12
:1071700013D0104B1F221E706E1C0021300004F033
:107180006FFA01992200300004F03AFA3100200031
:107190002C70002F06D004F073FAFEBD064B1220AF
:1071A0001D68DCE704F014FBF7E7C0467564FF1FB9
:1071B0009464FF1F1843FF1F9064FF1FF8B50F4E24
:1071C00012243368002B17D01B780F3C834213D155
:1071D00000250B4F0221387804F0F2FC094B042102
:1071E00038781D8004F0ECFC074B28001D803368C4
:1071F0005C7004F0CDFC04002000F8BD7864FF1F33
:10720000A064FF1F8C64FF1F7264FF1F70B501280C
:1072100023D11B4C2388002B03D01A4A1578002D4C
:1072200007D0194B1B68002B02D01878FFF7C6FF58
:1072300070BD3B2B02D93C3B2380F9E7134E022162
:10724000307804F0BDFCFA222388920002215A43D0
:10725000307804F03DFA2580EAE70B4B1B68002BE1
:10726000E6D00B4B1B785B07E2D5084B0221187860
:1072700004F0A6FC0022024B1A80FFF769FED7E754
:107280008C64FF1F7064FF1F7864FF1FA064FF1FE2
:107290007564FF1FF8B51E4D2868002803D004F060
:1072A000C7F900232B601B4E3068002803D004F080
:1072B000BFF900233360184F05243B7818002040A5
:1072C000234221D0154800F02BFA3B78234213D0FB
:1072D000202004F0EDF92860002813D0202200219E
:1072E00004F0BEF9202004F0E3F9041E306005D05C
:1072F0002022002104F0B4F9002004E0286804F002
:1073000097F92C601320F8BD00F00AFAF4E7C046A4
:107310009464FF1F9064FF1F7564FF1F0C43FF1FE1
:1073200010B50A4C23681A1E0ED0002808D101306F
:10733000587004F02DFC002805D02368002B02D0E3
:107340000021FFF787FE0122100010BD7864FF1FA7
:10735000F7B5274E050033680191181E21D05C78DF
:10736000244F012C30D1FFF7FFFD002825D020004D
:10737000FFF7F8F80400412814D91F4B02211878B0
:107380001E4A04F04DFA1E4B3C3C1C80022233681E
:107390005A703B78002B14D128000199FFF75AFE50
:1073A0000120FEBDFA2292004243002AEED0124B89
:1073B0000221187804F08CF9E8E7FFF7D3F802000F
:1073C000F3E700233B70EBE73B78002BE8D1032089
:1073D00004F0E6FB011E08D0D0230370CC3B4570BF
:1073E00083703368187804F013FCFFF7B1FDD7E71A
:1073F0007864FF1F7064FF1FA064FF1F60EA000035
:107400008C64FF1F10B51749838802008B4220D07F
:1074100011D815498B4217D0144900205B1899B236
:10742000012907D8926811785A425341D8B2FFF720
:10743000F9FD012010BD0E4A00209B1807229BB2C7
:107440009A424041C0B2F5E783681878FFF768FFB9
:10745000F0E7836899785A78090218781143FFF7A2
:1074600077FFE7E70A20000006200000F8DFFFFFB3
:10747000AFDFFFFF014B18707047C0461943FF1F75
:1074800010B5064C207001F041FA207804F070FB32
:107490000521207800F062FD10BDC046A064FF1FEA
:1074A0000BB273B50D00002B00DBC4E0884B1878DD
:1074B00004F0AEFA041E0ED00378912B0FD0A22B4D
:1074C00000D1A1E0834B1878FF2852D0210004F0AE
:1074D0009FFB00284DD180200002684076BD437894
:1074E0000F2B76D013D8052B70D00E2BEAD18088C5
:1074F000794B98422BD8794B98421BD8784B9842BD
:10750000E0D1A3681878591CFFF774F838E03E2BD7
:10751000D8D18378032B74D06CD8012B6ED0022B7A
:10752000D0D1704B1B68002B23D05B68002B20D080
:1075300098471EE06C4BC0180C28C3D804F008FA1A
:107540001DC2C2150BC20B0B0B3223C23C00674B92
:10755000C0180728B6D8664B1B68002B09D01B68DB
:10756000002B06D0200098470AE0A3681878FFF7A0
:10757000C7F8200004F064F8ADE7A068FFF762F8F0
:1075800000289FD0F5E7A3681B78002BF1D0554B5E
:107590001B68002BEDD01B68002BEAD0210055485A
:1075A0009847EDE74F4B1B68002BE2D01B68002B80
:1075B000DFD021005048F3E7504B1B68002BD8D098
:1075C0005B68002BD5D021004348E9E7FFF7EAF9D3
:1075D000CFE780884A4B984203D04A4B984200D06C
:1075E00070E7464B1B68002BC3D05B68002BC0D0F4
:1075F0002100D5E7153B012BBBD963E7FFF798FACC
:10760000B7E7FFF77DFAB4E73F4B1B78042B07D1B0
:1076100000236A4613800179408800F0C5FCA8E782
:10762000364B1B68002BA4D05B68002BA1D0010057
:10763000364898479DE7012421420AD0294B1B6810
:10764000002B04D05B68002B01D00020984701205C
:1076500043E78B070AD5264B1B68002B04D05B68D9
:10766000002B01D020009847022036E70421280093
:1076700008400D4200D131E7254E3388002B21D040
:10768000013B9BB23380002B1AD1FFF7DBF80028B7
:107690000AD0204B1C70164B1B68002B04D05B6873
:1076A000002B01D020009847FFF7C6F8694601F08B
:1076B00001FD6846FEF7FEFF1D20FEF753FF3080F8
:1076C00004200AE7024B187804F07AFAF8E7C0467B
:1076D000A064FF1F1943FF1F0E20000001200000BF
:1076E000091000009864FF1FFEDFFFFFAFDFFFFF00
:1076F0009C64FF1F0C2000000B2000008064FF1F13
:107700000D200000132000007564FF1FFFFF000024
:107710007264FF1F7064FF1F10B501F09BF910BD6C
:10772000014B18607047C0469C64FF1F0B88002007
:10773000162B01D817230420014A13807047C04636
:107740004A64FF1F00207047074A030011888142E6
:1077500007D091880020994202D101308000101892
:1077600070470020FAE7C046A864FF1FF0B58F7885
:1077700006000D00C5B01E2F15D1FFF7E5FF051E51
:1077800003D10024200045B0F0BD00223B003100B1
:10779000C078009200F0B2FB0400A81C00F0D2FBFD
:1077A000FF23EB70EEE7264B062403931B78FF2B99
:1077B000E8D0182FE6D87B08224A013BDB00029272
:1077C0009A589446002ADDD0029AD3185B68002BA1
:1077D000D8D00878002802D14B78012B02D106249A
:1077E000122FCFD107AFAB88697800976446AA689B
:1077F000A047041EC6D1AB78029A5B08013BDB00B0
:10780000D318390030005B689847041E0BD1AB7861
:10781000042BB6D0039A310010782200009700F0B4
:107820006DFB0400AEE76A78002AABD1AA7805A9FF
:107830003B88087130000A704B80FEF747FBA0E7D9
:107840001C43FF1FD8BD00111D4B37B505009842E2
:107850000BD000290AD1FFF777FF002805D119487E
:10786000FFF772FF002800D0058037BD01291AD12B
:10787000FFF76AFF041EF8D001235B420380A37860
:10788000FF2BF2D0FE2B07D00023E07814220093C8
:1078900029001E3300F032FBA01C00F053FB012333
:1078A0005B426380E1E70229DFD1013901F0BEF8D4
:1078B0000028DAD12800FFF747FF041EDFD1D4E704
:1078C000FEFF0000FFFF0000022210B5074B5242EE
:1078D0001A80074801325A809A80DA8000F07EFAD6
:1078E000044801F025F8002010BDC046A864FF1F21
:1078F0006D770011497800110388F7B50400002B5B
:1079000002D102252800FEBD4268022113782548D5
:107910005268FEF7A5FD00282ED0234F01253A8896
:10792000002AEFD0802321885B0201259B1A99420F
:10793000E8DC0C2003F0BCFE061E31D03B88228818
:107940009C4600231800019561469DB2491989B2F1
:10795000AA421BD8002801D062443A80002330009C
:10796000082208C0210003F04BFE104A1368002BC8
:1079700013D100251660C5E76268022113780C4810
:107980005268FEF76DFD0028C7D1BAE760681D0197
:107990004019418101330198D6E71A001B68E6E7D8
:1079A0001325AFE746BE00111A43FF1FA464FF1F53
:1079B00044BE0011014B18707047C0461C43FF1FA6
:1079C00014230A0010B51A40194204D001221021D4
:1079D00001F048F810BD4B06F9D40120884340005F
:1079E000F8E710B514008B0604D50122102101F030
:1079F00039F810BD08230A001A40194202D14BB2CF
:107A0000002B0FDA102101F02DF8002808D02300F8
:107A1000F2331B78002BECD0F1342378012BE8D122
:107A20000020E6E703208907FAD4E2E7F0B51F005B
:107A3000184B85B01C68019002910392002C27D14D
:107A4000200005B0F0BDA5683301ED186B89019ADF
:107A5000934211D3029A93420ED8002F04D10A9B6D
:107A6000002B10D12C00EBE73B002978039A6868C3
:107A7000FEF7F6FC0028F2D10136B6B2A388B34275
:107A8000E1D82468DAE7A3680A9A5B891380E9E7FA
:107A90000026F3E7A464FF1F37B50C000A88498865
:107AA0000123914217D3002A15D0651D23792A009E
:107AB00002210A48FEF7D4FC102300280BD02379BA
:107AC0006188208800242A000094FFF7AFFF0A2372
:107AD000A04200D0230018003EBDC04646BE0011A3
:107AE00013B50A0008884988012388420BD800286A
:107AF00009D00024137905320094FFF797FF0A2379
:107B0000A04200D02300180016BD13B50A00088853
:107B10004988012388420BD8002809D00024137912
:107B200005320094FFF782FF0A23A04200D0230011
:107B3000180016BDF0B58BB003904A8808880E0077
:107B40000123824255D3002853D00023012704ACDF
:107B500023700022718813000092FFF767FF051E53
:107B60003ED02078002835D12B78022B18D16770B1
:107B70006A8983000130E31880005A806968022214
:107B8000201803F03DFD23780133DBB22370042B72
:107B900019D93B006889013080B2002BD9D01FE091
:107BA00002236370122358436A89231804305A80D1
:107BB00069681022201803F023FD23780133DBB21B
:107BC0002370002BE5D10C4A6B899B185A42534114
:107BD000DBB2DFE76378012BE4D12B78022BC7D02F
:107BE00022780A23002A04D021000398FEF798F98E
:107BF000002318000BB0F0BD0100FFFF0F4BF0B5E4
:107C000004001868002816D083685D89A54207D84B
:107C10008288AE18B44203DA12019A18934201D155
:107C20000068EFE71E005F891036A74204D10029E3
:107C300000D00D801800F0BD3300EFE7A464FF1FF3
:107C400070B505000C0008880021FFF7D7FF03007E
:107C50000120002B04D022002800197AFFF7C1FE72
:107C600070BDF7B50C00002501902300EE331B78A2
:107C7000AB4201D800200AE06B00E65A0021300038
:107C8000E718FFF7BBFF002802D126800130FEBDB8
:107C9000017A0198FFF794FE002802D03B882380E8
:107CA000F5E70135EDB2E0E710B5040008880021E2
:107CB000FFF7A4FF03000120002B03D02000197A56
:107CC000FFF77EFE10BD0000054B1B68002B01D1A5
:107CD000180004E09A6852898242F6D19888704769
:107CE000A464FF1FF0B50E27002687B0039302ABF4
:107CF000FF183E8005001F4B40891400984207D0B2
:107D00002B78013000976A6880B2FFF78FFE06007B
:107D100002212B7818486A68FEF7A2FB00280FD0D2
:107D20006C892000FFF7D0FF002802D0013C041925
:107D3000A4B2039B002B00D01C80300007B0F0BD24
:107D400002212B780D486A68FEF78AFB0028E7D1EC
:107D500002212B780A486A68FEF782FB002807D0C8
:107D6000002EDED03B88A342DBD17489013CDFE7E3
:107D70006C89DEE7FFFF000046BE001144BE001123
:107D800042BE001110B50C00FFF7DEFC030002201C
:107D9000002B0AD0002C00D023609B781720FE2BEC
:107DA00003D00138FF2B00D1002010BD73B50D00AA
:107DB00001A904001600FFF7E5FF172805D0002EE3
:107DC00004D129002000FEF727F976BD01221021F9
:107DD000200000F047FE0028F3D0F6E7014B1860C2
:107DE0007047C046B464FF1F37B56B469D1D010048
:107DF00004000222280003F043FE2B88B02B0ED192
:107E00002379122B09D12300FA331B78012B06D1D9
:107E10000121608800F0E0F801E01B2BF8D037BDAD
:107E200010B5054B0421187000F098F8FFF74CFDD1
:107E3000FEF770FB10BDC046B864FF1F0020F0B510
:107E40000BB20F0087B0834234DA274B187803F067
:107E5000DFFD051E2BD00378A02B25D103AE31000A
:107E6000FEF7E4F8041E0BD1B378DB0724D51F4BD3
:107E700006341B68002B03D0310068889847040043
:107E8000A868002801D003F08BFC002C08D1184A08
:107E9000039B1340174A934206D0B3781B2B03D0A1
:107EA0000121688800F098F8280003F0C9FB8020C1
:107EB0000002784007B0F0BD0F4B1B68002B10D0BC
:107EC000310068889847041EDAD07378002BD7D128
:107ED000B27801A90A704B800C716888FDF7F6FF33
:107EE000CEE70624F1E7C046B864FF1FB064FF1F69
:107EF00000FFFF0000011200B464FF1FF7B50190FE
:107F0000FC200D0017001E0003F04AFE04001320A1
:107F1000002C12D0B02320002370089BF42267703D
:107F2000658026710830002B08D0190003F068FB2B
:107F30002100019803F06CFE0020FEBD089903F0BB
:107F40008FFBF5E710B5041E06D00078FD2803D896
:107F500003F036FCFF23237010BD00000A1F93B20C
:107F600010B504000220032B05D882400020024BEC
:107F7000D1529B189C7010BDD864FF1F0B8870B540
:107F8000043B04000D000220032B0BD8012120002C
:107F900000F04CFD03001420002B03D0290020002A
:107FA00000F0DEFB70BD000007B51300034A00922D
:107FB0000A00012100F02CFC0EBDC046E581001135
:107FC00007B5019203220092024B0A00122100F031
:107FD00049FC0EBD6382001107B56B4601AA1180F2
:107FE0000449D88008780633012802D1190003F02B
:107FF0008FFB07BDB964FF1F0C4B10B51870002331
:10800000FF210B4A1380138193819380094A538087
:108010001370517293819372D174D3821375517717
:1080200003F07EFC00F0FCF910BDC046E864FF1FC1
:10803000D864FF1FBA64FF1FF0B58DB06B460020F7
:1080400003910C229B5E834200DBB0E05D4B18780D
:1080500003F0DEFC051E00D1A4E00378902B00D0D5
:108060009DE006AF01004688380000F013FA7968F9
:108070000400002900D19CE03B88052B6ED13B8990
:10808000032B1CD905AC200000F0A2F86288172A47
:1080900061D83989131D994231D179682378043127
:1080A0000291D90738D5607800F08EF9071E06D006
:1080B000002303712378012B08D0132B23D0A86849
:1080C000002800D178E003F06BFB75E0628802992C
:1080D00009A800F0A6F80290380000F08BF909AA70
:1080E0002378387A0192002231000092029A00F03F
:1080F00012F9380000F064F9029B002BDFD0300049
:1081000000F080F9DBE70378032BD8D1628802996D
:1081100009A800F0D6F8DEE7122B13D1029909A8BE
:1081200000F0B5F8021EEAD127498B88002BC6D093
:10813000887909A92378019161780091310000F0D4
:10814000EAF8BCE7002302AA93833000617809AA09
:10815000FFF72AFFB3E71D4B0993F6E7042B02D084
:108160009A1F012AABD8184A043B9B00995A002950
:10817000A5D0D218907831003A0000F0AEF800286F
:108180009DD13B88042B03D001213000FFF724FF51
:10819000012C04D1A868002801D003F001FB2800BD
:1081A00003F04EFA8020039B0002434018000DB0FC
:1081B000F0BD012800D182E701213000FFF70CFF5C
:1081C000EDE7C046E864FF1FD864FF1F01001700F9
:1081D0000B7803704B784370CB788A781B0213437B
:1081E000438070470A88030002700A88120A4270AE
:1081F0000A88012A06D14A8882704A88120AC27007
:108200000420704702208242FBD14A8804309A70D1
:108210004A88120ADA708A881A718A88120A5A7190
:10822000EFE710B50400012082420CD94B780A78A0
:108230001B0213432380834206D1CB788A781B022A
:1082400013436380002010BD022BFBD1CB788A78CA
:108250001B02134363804B790A791B021343A380EB
:10826000F0E70B8803700B881B0A43704B88837000
:108270004B881B0AC3708B8803718B881B0A437160
:10828000CB888371CB881B0AC37108207047030019
:108290000120082A14D14A780878120202431A8071
:1082A000CA788878120202435A804A790879120201
:1082B00002439A80CA798879120202430020DA8048
:1082C000704710B504000120022A05D100204B7828
:1082D0000A781B021343238010BDF8B50600102056
:1082E0000F00150003F05CFC04000120002C0ED0F0
:1082F000A0230C22290023806780201D002D07D099
:1083000003F07EF92100300003F082FC0020F8BD6C
:1083100003F0A6F9F6E7F7B51E00009008AB1420AD
:1083200017001D78019103F03BFC041E12D0A2231C
:108330000370019B47704380099B057146710C22B5
:108340000830002B07D0190003F05AF921000098DB
:1083500003F05EFCF7BD099903F082F9F6E737B543
:10836000041E0FD04388002B0CD00025C188132396
:10837000007A172201950095FFF7CDFFFF23658056
:108380006372257037BD000010B50C4904004A889F
:10839000002A09D08B89002B05D00020CB8A02222D
:1083A000834201D010BD012213000A204343002064
:1083B0004032C854C81842800472F3E7BA64FF1F01
:1083C0000023438003707047094B00211A0010B549
:1083D0005C88002C06D01C79844203D10A234B43CD
:1083E000D01810BD01310A330329F1D10020F8E77C
:1083F000BA64FF1F10B50400407A03F0E1F9FF23CF
:10840000637210BD7047043010B580B203F0A8FA53
:10841000002803D00421494203F0CAFB10BD00002C
:1084200070B50025104CA0682580A581A580A842C4
:1084300002D003F0B5F9A56000250C4C0C4B606D23
:108440001D80230058331D70A84202D003F0A8F904
:10845000656500256068002801D003F0A1F90135A9
:1084600008340A2DF6D170BD8065FF1F2465FF1FFB
:108470007465FF1F70B5041E09D1054D2880A881C1
:10848000A880A868002802D003F08AF9AC6070BD0B
:108490008065FF1FF0B54B8885B0019300234360D2
:1084A0000A7905000F00022A00D07BE0CA88032A5F
:1084B00017D98B685E7819783602DC78D8790E4344
:1084C00099781B7A24021B020C43034353495BBA7D
:1084D0000B80331D93421ED1042C04D0631F022B4A
:1084E0000ED9012015E0019A4D4B1201D35A002BF1
:1084F00006D00198FFF7BEFF4A4A136901331361A2
:108500000421B8682E812C80494203F051FB686039
:10851000002005B0F0BD434D042C06D0631F022B94
:108520000FD9EB680133EB60DBE7019A3C4B12019A
:10853000D35A002B05D00198FFF79CFF2B6901331C
:108540002B61374B30000293019B029A1B01019370
:10855000002301998C468B52130063449C80039343
:108560009E81FFF750FF039B041E986016D00421E4
:10857000B868494203F01CFBFA880100043A200065
:1085800003F03EF80199029AFB888A5A043B9B1833
:10859000029A8B522B6801332B60A2E7AB6901333F
:1085A000AB619EE71E4B0293019B1E01029BF35A97
:1085B000002B2DD002998C19A068002828D0012A00
:1085C00026D1FA889B189BB27352A189994217D37E
:1085D0009B1AC018B96803F013F8029BA289F35ADA
:1085E000934200D07DE700222B81A3882B80A368D3
:1085F0006B60029BF2520B4A53680133536070E781
:10860000084A9368013393600198FFF733FF68E7E6
:10861000044A536901335361F6E7C046EA64FF1F19
:108620008065FF1FF064FF1F70B5051E15D10B4C50
:108630000B4B1880230058331870606D002802D04F
:1086400003F0AEF86565250050356068002801D05C
:1086500003F0A6F80834AC42F7D170BD2465FF1FC3
:108660007465FF1FF0B51700A12285B09200019339
:108670004243394B06001B680C009B18D933FF336B
:108680001D78FDF741FF0430854204DD3000FDF721
:108690003BFF0430C5B2BD4207D33A000021300091
:1086A000019B02F0FDFF05B0F0BD2900380003F08A
:1086B000D7F82300C6B250331E700393019B2900E4
:1086C0006365380003F08CFACBB20293002B02D022
:1086D000039B01361E7000262300503303931B7842
:1086E000B34204D8606D002831D10020DBE7029A44
:1086F0002800002A04D0013B1000B34200D028001B
:10870000F700E719387003F033F8786000280ED0CE
:108710003A78019902F074FF019A3B780136D31838
:108720000E4A0193D369F6B20133D361D4E7039BB8
:1087300018706065A74205D1084A1320D36A013337
:10874000D362B0E7606803F02BF80834F2E703F077
:1087500027F800236365C8E73409FF1FF064FF1F93
:10876000F7B50D0007000421686803F021FA2B8992
:10877000040003702B891B0A43702B8883702B889D
:108780001B0AC3702E8902250436F6B2F42E15D8C2
:108790001B4B9F4214D10C2003F002FA1135011E2D
:1087A0000CD0902303708E3B0371043B4380154B28
:1087B0008460C680187803F02BFA00252800FEBDDF
:1087C0005C237B43104AD3180093583301931B78E2
:1087D000002B0FD10300320038000099FFF742FF51
:1087E000019B05001B78002BE8D13800009902F0AE
:1087F000CFFFE3E7054A0725536A01335362DDE7FC
:10880000FEFF0000E864FF1F2465FF1FF064FF1FE8
:10881000F0B587B0009017200F0016000193FFF706
:10882000F2FD1325041E19D00C98031E02D00199E5
:10883000201D9847030AE370052302AAA0700430A4
:10884000908127700098667003A993800494FFF7C5
:1088500087FF051E02D0200002F0A2FF280007B00B
:10886000F0BD0000F0B587B01F000CAB1B78039182
:10887000059301210DAB06001C78049200F0D6F898
:108880001425002821D02000FFF77EFD0135041EAD
:108890001BD01149059B0A7803700132D2B2131E16
:1088A000C68001D101231A000B7022713000049B95
:1088B00003990097FFF7ACFF051E09D123002100A3
:1088C0000648074A093303F0C3F8280007B0F0BD93
:1088D000002363802370F8E7EC64FF1F5F830011BF
:1088E00030750000F8B505000E00064C064F2368F1
:1088F000002B02D03100280098470434BC42F6D146
:10890000F8BDC0469065FF1FA465FF1F0123064AFE
:108910005B425380002313715362044A1360536017
:108920009360D36013617047A465FF1F9065FF1FBC
:108930000200002310B506499C000859002801D107
:10894000625010BD0133052BF6D11320F9E7C04664
:108950009065FF1F034A5388181A4342584140420A
:1089600010407047A465FF1FF0B585B002930AABB5
:108970001F780CAB1B88009008000E000192039337
:10898000FFF7E8FF05001120002D1BD10E48FFF76F
:10899000E1FF04001520002C14D006220B99A771CA
:1089A000E01D02F02DFE019B30002371029B290087
:1089B0006371009B66802370039B6562E381FFF710
:1089C00091FF280005B0F0BDFFFF000010B5FFF7D4
:1089D000C1FF04000220002C12D060880121FFF7A3
:1089E00081FF606A002801D002F022FE28220021C7
:1089F000200002F035FE012300205B4263802071DD
:108A000010BD000030B5074A074C558801001378A7
:108A10000020A54204D05B1A59424B4158421040F5
:108A200030BDC046A465FF1FFFFF0000084A10B517
:108A300001230C00904208D0FFF78CFF031E04D0E6
:108A4000037923405A1E9341DBB2180010BDC04683
:108A5000FEFF0000024B1879431E9841C0B27047D8
:108A6000A465FF1F70B504000D001600FFF772FF2C
:108A7000002804D10D4B9C4200D0143070BD416AD7
:108A800003790520002907D012221A40102A02D1AA
:108A90000520002EF2D10F20DB06EFD5897E0C20B9
:108AA000A9428941494249420840E7E7FEFF0000E8
:108AB000030010B5002800D110BD0348034A4188C7
:108AC0009142F9D09847F7E7A465FF1FFFFF000028
:108AD000002330B5C45CCD5C6C40D4540133102B02
:108AE000F8D130BD0F23002210B5C45C64002243CE
:108AF000CA54C25CD209013BF7D210BD020001008A
:108B000010B52032103102F06BFD10BDF0B58BB006
:108B10000390102005931700049102F0C9FD009006
:108B2000102002F0C5FD009B13240190002B05D0FE
:108B300000280CD11324009802F07AFD019B002B31
:108B400002D0180002F074FD20000BB0F0BD102020
:108B500002F0AEFD0600102002F0AAFD132405006D
:108B6000002E00D1AEE0002819D01022002102F022
:108B700077FD32002900039802F032FD041E0ED169
:108B800033787F2B51D830000099FFF7ABFF009B63
:108B90001B787F2B53D801990098FFF7A3FF300073
:108BA00002F046FD002D02D0280002F041FD002C0D
:108BB000C1D1102002F07CFD0600102002F078FDEB
:108BC0000290002E7CD0002878D03A000F3223008B
:108BD0000125121105D00F333B4015B25A425341C3
:108BE0001BB26A1E1201002B33D0049BD2B298181C
:108BF0000099029AFFF76CFF013D1022002130001E
:108C000002F02EFDADB2049F2D017D19AF4242D07E
:108C1000002C33D0300002F00BFD029B002B00D162
:108C200089E7180002F004FD85E729003000FFF70E
:108C300059FF28002549009AFFF74AFFA7E72900B6
:108C40000098FFF74FFF28002049019AFFF740FFE7
:108C5000A5E70F210F4004998A18D9B28F4208D98D
:108C6000D15C06A819540133102BF6D1029A019950
:108C7000C0E7791A48424141C901F2E739003000A2
:108C800006AAFFF725FF3200039806A902F0A8FC08
:108C900010370400BAE7002CBCD13000029906AAB4
:108CA000FFF716FF320006A9039802F099FC08228C
:108CB00004003100059802F0A3FCABE71324A9E7F8
:108CC0001324AAE7002800D06EE733E74CBE00115A
:108CD000F0B58BB00F0016000225009000283FD0A1
:108CE000002A3DD00B1DDBB21800029302F0E0FC1D
:108CF0001135041E34D0FDF747FD05003A000099F8
:108D0000201D02F0A5FCEBB20393E3702B0CDBB249
:108D10002F0A00936370FFB22B0E2370A77001938C
:108D2000FDF72CFD1022010006A802F091FC2100A5
:108D3000029A04AB06A8FFF7E9FE051E0DD1039BBE
:108D400008223370009B04A9B370019B7770F37005
:108D5000301D02F07DFCFDF71DFD200002F068FCD7
:108D600028000BB0F0BDF0B58FB00D00149E03903D
:108D700004920593002A03D1022420000FB0F0BD15
:108D8000002EF9D00398FFF7E5FD1424071EF4D058
:108D90007278337812021A43B3781B041343F278C3
:108DA00012061A43036A0192934201D30133E3D1BD
:108DB000002D03D03B7901249B07DED5082200213A
:108DC00006A802F04DFC059B13240433DBB2180007
:108DD000029302F06DFC051ECFD0059A0499043071
:108DE00002F036FC04223100280002F031FC390088
:108DF000102210310AA802F02BFC2900029A06ABBF
:108E00000AA8FFF783FE041E0FD1082206A908A8AE
:108E100002F01EFC0822311D08A802F071FE012894
:108E200007D101990398FDF7C9FC280002F000FC66
:108E3000A3E70124F9E7000070B51C4C0500236886
:108E4000181E10D0002D14D11A78002A0CD1981CAD
:108E5000083202F0D5FB02F0DBFC0135002808D116
:108E600023681D70012070BD0A331800082202F02B
:108E7000C7FB2368002BF5D0122002F091FE061EDE
:108E80000DD0C123216803704570023110220230D9
:108E900002F0B6FB23683100587802F0B9FE206872
:108EA00002F0C6FB00232360DCE7C046CC65FF1F51
:108EB000F8B504002020FDF755FB0D4EA700BB5967
:108EC0000500002B0DD000280BD0D878FF2809D141
:108ED00008492A000C55F35907480333611802F07A
:108EE000B7FDF8BD290002F0CBFC0028F0D1F8E76F
:108EF000E865FF1FD065FF1F09A1001170B5064D81
:108F000084006359002B05D0D87802F059FCFF2269
:108F10006359DA7070BDC046E865FF1F70B5060082
:108F20008CB00C00150000213022684602F098FB3E
:108F300031001022684602F08BFB1D202100032225
:108F4000684402F085FB6846FFF7D8FD2D21040038
:108F500003222800694402F07BFB20000CB070BDA6
:108F6000F0B50700160097B001931CAB1D783022B6
:108F70001EAB00910AA800211C7802F071FB1022A0
:108F800039000AA802F064FB1022002102A802F0B6
:108F900067FB0722310002A802F05AFB072202AB4E
:108FA0009818631E9C41019902F052FB02AB9C731E
:108FB0002B005A1E934102AAD3730021102206A847
:108FC00002F04EFB06221D9907A802F041FB1A2071
:108FD00002ABC01806221F9902F03AFB102200993A
:108FE0000EA802F035FB102202AB0EA908781C78FF
:108FF000013A6040D2B2087001330131002AF5D144
:109000000AA8FFF77BFD102212A904000EA802F0A7
:10901000F7FA102206AB0EA908781D78013A6840CD
:10902000D2B2087001330131002AF5D10AA8FFF746
:1090300065FD044310222098E4B212A902F008FB57
:10904000200017B0F0BD70B50E0014008CB0010008
:10905000102268461D0002F0FBFA3100082204A825
:1090600002F0F6FA2100082206A802F0F1FA68469A
:10907000FFF744FD04001022280008A902F0E8FAD6
:1090800020000CB070BDF8B506000D0000243719A3
:10909000AC4200D3F8BD02F0A3FC030A3B70631C92
:1090A000DBB201379D4203D90234F054E4B2EEE75B
:1090B0001C00EDE773B506000C000225002819D04E
:1090C000002917D0032101A8FFF7DDFF6B469A792D
:1090D0003F231A40013313436A463000937101A9BC
:1090E0002200FFF71BFF051E04D10322E01C01A98B
:1090F00002F086FA280076BD03785807DA08C00F18
:10910000D20080009B0710439B0F1843C0B27047EA
:1091100007230B40C908C9000B43037070470000C8
:1091200070B50400FFF7EAFE134DA4006359002B4D
:1091300021D0186A002801D002F07AFA2B59986ED3
:10914000002801D002F074FA2B59D86E002801D003
:1091500002F06EFA2B59186F002801D002F068FA5D
:109160002B59586F002801D002F062FA285902F0FA
:109170005FFA00232B5170BDE865FF1F0E4B800086
:10918000C35870B50C00002B0FD09D68002D0CD07B
:109190002B78201D0B706B784B70A97CFFF7B8FF04
:1091A0002B7E23726B69E36070BD102200212000CA
:1091B00002F056FAF8E7C046E865FF1F014B186059
:1091C0007047C046E465FF1F074A030080008258CD
:1091D00010B5002A06D0D088984203D1012901D1C8
:1091E000FFF79EFF10BDC046E865FF1FF0B5264E95
:1091F00095B087000B93BB590500099112200A9284
:10920000002B31D0D888FFF7A5FB04001420002CD8
:109210002AD0280010A9FFF7B1FFBB591E781D6A9C
:10922000002E23D00895FDF7EFFA07000020FDF788
:10923000F1FA0790A379E61D069310AD0CA90898E2
:1092400000F0E2FA0EA9280000F0D7FA0B9B0A9969
:109250000493069B09980293079B0396019300973A
:109260000EAB0CAAFFF77CFE15B0F0BDFDF7CCFAF3
:1092700006903000FDF7CEFAE31DA779079310ABF7
:1092800006000893DAE7C046E865FF1F30B50C4CCE
:1092900085002A59030085B00120002A0ED018004D
:1092A0006946FFF76BFF2B591A78D888054B002ABF
:1092B00000D1054B6A46072100F0D9FB05B030BD4F
:1092C000E865FF1FFB9700110998001130B5094CA4
:1092D0008500295985B010226846253102F090F9A1
:1092E0002A591121044BD0886A4600F0C0FB05B012
:1092F00030BDC046E865FF1FA598001130B5094C88
:109300008500295985B010226846353102F078F978
:109310002A591121044BD0886A4600F0A8FB05B0F9
:1093200030BDC046E865FF1FE3980011F7B54D4F0B
:1093300086001020F4590D0002F0BAF9F3592062AA
:10934000186A132200286CD0033A29009C6802F0A6
:1093500057F9F3591A780192002A58D11E6A227DD2
:10936000317B944651400122019F114201D1674651
:109370001740217D914339432175377B4F40BC46CF
:1093800060460027800701D44F08174001210220C2
:109390008F40227D82433A432275377B5740BC463B
:1093A00060460027400701D497080F400420227D23
:1093B000BF0082433A432275627D0027944660468F
:1093C000727B42400A4201D167460F400121627D13
:1093D0008A433A436275777B5740BC466046002714
:1093E000800701D457080F400220627D7F0082432E
:1093F00017436775767B00227E40760701D4BA0852
:109400000A400426617D9200B1430A4362756A787E
:10941000002A08D06278002A05D005220533DA77C1
:1094200000221000FEBD04222979114205D1A17C41
:10943000114202D10533033AF1E7019A21782C78E1
:10944000002A02D10A002100140018220429E8D8B9
:10945000042CE6D805206043034A05331218525CF9
:10946000DDE7C046E865FF1F5CBE001110B50A00CD
:109470001121024B00F0FBFA10BDC0463F990011CC
:109480000B0030B587B001AD2B806B460400110096
:10949000981D082202F0B4F82A000B212000024B8C
:1094A00000F0E5FA07B030BD6799001110B50A0069
:1094B0001121024B00F0DBFA10BDC046BB99001130
:1094C00013B50B0011006A4613706B4604000622A8
:1094D000581C02F095F86A4608212000014B00F064
:1094E000C6FA13BDDB99001110B50A001121024B19
:1094F00000F0BDFA10BDC0462B9A00117FB50500E3
:109500000B4BAA00D4580800002C0FD0666F237FA5
:10951000E28821780396266F0296E66E0196A46E85
:109520000094FDF709FC2800FFF7FAFD7FBDC04657
:10953000E865FF1F10B51721FFF7E0FF10BD000021
:1095400070B50A000D00064B0221040000F08FFAEE
:10955000060029782000FFF7D1FF300070BDC0461B
:109560000B99001170B586B000236A4613708368AA
:1095700004001D78681E0A2859D801A902F000FBD2
:10958000060633373B3F43474B4F5300180000F06C
:1095900042F9062312284BD000281BD16088FFF720
:1095A000D9F90823002813D04279002A47D1264B45
:1095B0001A78072312070BD5244B1A680723002AB1
:1095C00006D01668002E03D0290001AAB047030078
:1095D0006A4613706B461B786088002B2AD1FFF710
:1095E00067FC06B070BD180000F06CF9D4E71800F5
:1095F00000F087F9D0E7180000F093F9CCE71800E5
:1096000000F0ADF9C8E7180000F0C3F9C4E718008E
:1096100000F0F6F9C0E7180000F0F6F9BCE7180012
:1096200000F013FAB8E7180000F013FAB4E70723C4
:109630006A46137069466088FFF782FFD1E7052309
:10964000012AC5D1024BB8E77564FF1FE065FF1F13
:10965000E465FF1FF8B52C4F8600F35904000D0098
:10966000002B40D0DA8882423DD15A78062A33D185
:109670001A78002A2ED0012099681A6A097D0142C1
:1096800006D0157B054203D007225A700120F8BD91
:109690000220014204D0157B054201D00922F4E7E3
:1096A0000420014204D0127B024201D00B22ECE7DD
:1096B000164B1B68002BE9D05B68002BE6D020001E
:1096C0009847BB5900215B78122BDFD12000FFF7B0
:1096D00015FFDBE70E4BECE7112A04D1002900D07F
:1096E00032252900F2E7002D08D12000FFF732F9DA
:1096F000002803D0102302791343037121002800AE
:10970000FDF798FAC2E7C046E865FF1FE065FF1F56
:10971000E465FF1F70B50E4E8500AB590400002BA9
:1097200013D01B78002B11D10A4B1B68002B04D0DF
:109730005B68002B01D02000984773595B78122B8F
:1097400003D100212000FFF7D9FE70BD024BECE7EA
:10975000E865FF1FE465FF1FE065FF1F094B800000
:10976000C3581020002B0CD01A6A002A09D09B681D
:10977000002B06D0127A1B7E101C9A4200D9181CAE
:10978000C0B27047E865FF1F70B503000D001400FC
:109790000220002A30D000292ED013700B78081D2B
:1097A00053704B789370FFF7A7FCE0700120022103
:1097B0002B7A23716B7B034063716A7B0A401343EE
:1097C000042263716E7B1640334363716E7BF6082F
:1097D000F600334363712B7B0340A371287B014068
:1097E00000200B43A371297B0A401343A3712A7BFA
:1097F000D208D2001343A37170BD10B50A00010056
:109800000120FFF7C1FF10BD10B50A0001000220C2
:10981000FFF7BAFF10BD70B506000C000220002E45
:1098200030D000292ED07378201D0B70B3784B7088
:10983000F178FFF76DFC01223579257271794B10B3
:1098400008001340934010400343881010408000EC
:10985000C9080343C9000B436373B1794B10080077
:109860001340934010400343881002409200C908FF
:109870001343C9000B4321202373FCF773FE854279
:1098800001D2122070BD2220257AFCF76BFE8542A2
:10989000F7D823781820042BF4D86378012BF1D85B
:1098A0000020EFE7030010B50220002909D0002BAB
:1098B00007D00322481C0A7019000D3201F0A0FEE7
:1098C000002010BD03000222080010B5002B06D0B6
:1098D000002904D00E32591C01F092FE0022100023
:1098E00010BD030010B50220002909D0002B07D0BD
:1098F0000422481C0A7019000C3201F081FE00207D
:1099000010BD10B5FFF7DEFF10BD030002200029D7
:1099100006D0002B04D0052200200A701B784B7063
:10992000704703000220002B08D0002906D05B7886
:1099300000200B70013B082B00D918307047030042
:1099400010B50220002909D0002B07D00622481CA0
:109950000A7019000A3201F053FE002010BD10B544
:10996000FFF7B0FF10BD02000B00022010B5002968
:109970000ED0002A0CD00721197011885970118857
:10998000090A997011180822D81C01F039FE00202C
:1099900010BD03000A00022010B5002B0CD00029D6
:1099A0000AD099785878090201431180901CD91C7B
:1099B000082201F025FE002010BD030010B5022092
:1099C000002909D0002B07D00822481C0A70190072
:1099D000921801F015FE002010BD02000B000220BD
:1099E00010B500290BD0002A09D00921197011786F
:1099F00018185970511C062201F002FE002010BDFB
:109A000010B5FFF75FFF10BD02000B00022010B57C
:109A1000002A09D0002907D05178197011180622A0
:109A2000581C01F0EDFD002010BD030010B5022010
:109A3000002909D0002B07D00A22481C0A701900FF
:109A4000063201F0DDFD002010BD10B5FFF73AFF32
:109A500010BD02000B00022010B5002A06D000291C
:109A600004D018005178FFF753FB002010BDF0B56B
:109A700085B017001E006A46062305000800918184
:109A80009380FEF7C0FC1324011E02900CD0380016
:109A9000B047041E05D1280001A9FEF76FFA041E85
:109AA00002D0029801F07CFE2800FFF701FA2000A6
:109AB00005B0F0BDF0B504008BB001911500002198
:109AC000102202A801F0CCFD334EA700B85900289F
:109AD0003CD0C388A34239D10378002B36D14278D9
:109AE000062A18D102000100553235310C3006AB80
:109AF000FFF7A9FA002829D12000FFF72FFE020066
:109B000006A902A801F07CFD200002A901F080FD59
:109B100001200BB0F0BD816E002917D00B8A112AED
:109B200028D19D420ED101981231093A01F0E8FF87
:109B3000012807D1BB5920009D6EFFF70FFE2900B9
:109B40000200DEE732212000FFF7D8FC2000FEF7FC
:109B500001FF061E1BD0416A002918D00B8AAB42B8
:109B600015D108220198123101F0CAFF01280ED147
:109B7000716A0AE09D42E9D108220198123101F090
:109B8000BFFF0128E2D1BB59996E8A7EB9E7200058
:109B900001F086FEBCE7C046E865FF1FF0B56B4DDF
:109BA00087007E5985B0337802900393002B00D054
:109BB00087E0B368346A01937078062817D10122D0
:109BC0001B7D134202D0217B114218D10222134285
:109BD00002D0217B114251D10422134203D0237BB6
:109BE000134200D08BE0019B5A7DEB5991E007387E
:109BF0000428F8D801F0C4FF032E42678300B36E37
:109C0000002B03D11C2001F053FDB066EB599C6E74
:109C1000002C1CD010220021200001F021FD029810
:109C2000FFF79CFD01002000FFF72DFA01F0D8FEA0
:109C30002082200008211230FFF725FA0298FFF752
:109C40008DFDA076EB592100D888FFF70FFC082284
:109C5000EB591CE0B36E002B05D01A00198AF0886E
:109C60001232FFF70DFC0222019B197DEB591142C4
:109C70003DD0207B10423AD0073208E0F488FCF750
:109C8000DBFD01002000FFF711FC0A22EB595A709E
:109C9000029B9C002A595378073B042B11D8D0888B
:109CA000FEF758FE00284ED0C3895A08D21828491A
:109CB000029B0298CB542B5941180433254801F0DC
:109CC000C7FE05B0F0BDFCF79FFD030001208342F5
:109CD00001D100200393EB59DE88FCF79BFD03992B
:109CE00002003000FFF7ECFB019AEB59117D0422D2
:109CF00011420CD0217B114209D00B22C7E7F68814
:109D0000FCF73CFD01003000FFF7EEFB6BE7019A2A
:109D1000527D01210A4204D0607B084201D00C220E
:109D2000B5E702210A4204D0607B084201D00E222E
:109D3000ADE704210A4204D0627B0A4201D010221E
:109D4000A5E71222A3E7FA225200B0E7E865FF1F59
:109D5000EC65FF1F13A1001110B5064B1A78042300
:109D6000100018401A4200D00348FFF727FA0020DD
:109D700010BDC0467564FF1F2043FF1F70B504006F
:109D8000FFF7D4FA051E43D12000FFF77FFA234ED8
:109D9000A400A0598268937CDB0708D50321036ADD
:109DA0001B790B40012B02D1017F0B430377431D2D
:109DB000D97F8B1E022B0DD8022900D00121C0882B
:109DC000FCF790FF042133591A7F59700A431A7720
:109DD000280070BD01290CD10223102243700021FC
:109DE0000C3001F03DFC305910213530FFF74BF9B4
:109DF000EEE70529ECD10223D118437010220C3074
:109E000001F0FEFB04233259117F0B431377EAE77D
:109E100008251828DCD1053DDAE7C046E865FF1FB4
:109E2000F0B58BB0059143887E4F9E00F459150024
:109E30000493002C15D1012902D000200BB0F0BDF5
:109E4000101D57781678FFF757F9EB683200029328
:109E50002B7A0499019300903B002000FCF70CFF43
:109E6000EBE7E388049A934201D00820E6E72378E1
:109E7000012B00D1D4E0059B581E092800D9CFE062
:109E800001F07EFE05CE0A29CC506C859AB22900DD
:109E90000498FFF773FFD1E7200029001022453016
:109EA00001F0AEFBB9594B78042B02D1013B4B704A
:109EB000C3E70B000A00253335320C310498FFF755
:109EC00095F90498FFF702FA0522431E9841BB5901
:109ED000C0005A70B2E7200029001022553001F06E
:109EE0008FFB049B4F4C9D00295904980A0006AB38
:109EF00055320C31FFF77AF929591022453106A85D
:109F000001F0FEFD012808D10498FFF7F7F905904C
:109F1000002804D106222B595A7005988EE7082391
:109F20000593FAE763780C2B7AD1E36E002B03D10B
:109F30001C2001F0BDFBE066BB59D86E00286FD035
:109F40001022290001F05CFBBB590498DC6EFFF77E
:109F500005FC0D22A076BB595A706EE7E06E002812
:109F60005ED063780D2B5BD12B8808220382A91C5D
:109F7000123001F045FBBB599A68517D0222114213
:109F800026D0186A407B104222D00C32E4E7637876
:109F90000E2B45D1236F002B03D1162001F088FB37
:109FA0002067BB59186F002803D01022290001F048
:109FB00027FB0F22BB59CFE763780F2B30D1206FDF
:109FC0000622691C103001F01BFBBB599A68517DB9
:109FD0000422114203D0196A497B1142D5D10021D4
:109FE0000498FFF78BFA28E7636F002B0DD0BB595D
:109FF000586F0028F3D01022290001F001FB012244
:10A00000BB5952425B6F1A61E9E7142001F050FB23
:10A01000BB5960675B6F002BE9D126E72978DFE742
:10A0200007200BE7E865FF1F10B5064C207001F014
:10A030006FFC06212078FDF791FF0348FEF778FCBE
:10A0400010BDC046FB65FF1FC991001100200BB277
:10A0500070B50D00834216DA264B187801F0D8FC53
:10A06000041E0DD00378922B0ED0A02B37D0224B9C
:10A070001878FF283AD0210001F0CAFD002835D118
:10A0800080200002684070BD43780E2B0BD03E2B21
:10A09000EDD18378052B12D0082BE8D18179808807
:10A0A000FFF7D8FA08E0154B82889A42DFD183681F
:10A0B0001878591CFEF7C0FE002817D1D7E7104BBF
:10A0C0001B785B0712D50F4B1B68002B0ED09B68CB
:10A0D000002B0BD0C289811D80889847ECE7FFF7E1
:10A0E00041FAA068002801D001F05AFB200001F0DD
:10A0F000A7FAC5E7FB65FF1F1943FF1F18200000E3
:10A100007564FF1FE465FF1F10B50078FFF712FAB2
:10A1100010BD10B50078FFF7FDFA10BD0C234343C6
:10A12000084A10B59B185A68002A03D0012901D1AA
:10A13000904710BD9B68002BFBD00029F9D19847B0
:10A14000F7E7C0461866FF1F01238340094A10B590
:10A15000946B1C439463506B98435063D46B200002
:10A160009843012901D120001843D063116B0B43A0
:10A17000136310BD00800040F0B500240127154B8B
:10A1800085B0DA6B144E03921A6C0192DA64019B6B
:10A19000E3403B4217D0039DE5403D400295E5B2C8
:10A1A00002992800FFF7BAFF316A736A002908D0C4
:10A1B0003900002B01D0029979402800FFF7C4FF35
:10A1C00001E0002BF9D101340C36172CDFD105B09A
:10A1D000F0BDC04600800040FC65FF1F064B01211A
:10A1E0005A68C2400A4204D01B68C34018000840A5
:10A1F00070471B6DF9E7C046008000400122064B06
:10A200008240002903D0D9680A43DA607047D968D0
:10A210009143D960FAE7C0460038004030B50324C6
:10A2200044430F4BE25C1B199C785D7801232D1B86
:10A230000135AB40013BA340A140DB430C00122899
:10A2400007D808499200521811681940214311603B
:10A2500030BD054A11680B4023431360F8E7C04640
:10A26000A3BE001108F0004014F00040C21F70B5FA
:10A27000D4B20623092C0BD80125084C954000299F
:10A2800008D00021FFF7CAFF23682B432360002377
:10A29000180070BD2368AB43F8E7C04600380040A3
:10A2A000214BF0B51B185B78022B21D103244443CA
:10A2B0001E4A1F4EA35C1219947801221500854096
:10A2C000B76B013CE4B23D43A240B563194C122880
:10A2D00015D89B0000290CD117495B1899680A43CF
:10A2E0009A600123205C154A834011680B43136078
:10A2F000F0BD11495B18996891439960F1E70E4BE5
:10A3000000290DD159690A435A61225C1328E8D00B
:10A310000123203A93400A49086803430B60E7E7AA
:10A32000596991435961F0E7FC65FF1FA3BE001115
:10A3300000800040E8BE001100F00040A0F00040A6
:10A34000A4F00040F8B500241B4E1C4D1C4B1B5DB7
:10A35000012B1FD1194A9269E2401A420BD0012207
:10A36000B25693402200143AD2B2022A09D81549B3
:10A370004A6913434B61013402360C35172CE5D181
:10A38000F8BD0022B2560F499200521891680B4353
:10A390009360F0E7022BEED1E7B23800FFF71EFF23
:10A3A00001235840C1B23800FFF77AFF3800FFF7A9
:10A3B00015FF6877DFE7C04675BE0011FC65FF1F1B
:10A3C000FD65FF1F00F00040012202388240054B6E
:10A3D000002903D059690A435A617047596991436A
:10A3E0005961FAE700380040F8B50E0001210F006E
:10A3F0008740114A0400D368FD43BB43D360831EEA
:10A400008B4201D8FFF7E0FF00212000FFF72EFF6D
:10A410000A4A0B4B5168012E05D139431B19516073
:10A420005E700020F8BD2940516002221C19627044
:10A430009A6915409D61F4E70038004000800040B3
:10A44000FC65FF1F012210B58240074B002906D092
:10A4500019680A431A600121FFF7C6FF10BD196889
:10A4600091431960F7E7C046008000400C2370B5A7
:10A47000002543430A4A29009B181D70094B04001C
:10A480001B185D70FFF7B0FF0123A34006492800A9
:10A490000A681A430A6005490A689A430A6070BD4F
:10A4A0001866FF1FFC65FF1F3480004030800040AD
:10A4B00070B504000E00FF2813D003250540FFF7F8
:10A4C000D5FF084AA3089B009B183F22ED00AA4035
:10A4D000AE40196820009143314319600121FFF714
:10A4E0008DFE70BD18380040F8B50C244443134B62
:10A4F0000500E4186368002B03D1A3681220002B29
:10A500001AD0022201270E4B00215B195A70280035
:10A510002770FFF769FF63681E1E08D0A3683E001E
:10A52000002B04D02800FFF759FE4640F6B2280061
:10A530003100FFF709FE0020F8BDC0461866FF1F76
:10A54000FC65FF1FF7B5C420FF222B4B8000195874
:10A55000002491433F3A0A431A508022274F520267
:10A56000274E1A60274B1D5D002D21D0A31E012B05
:10A5700003D80121E0B2FFF727FF012D18D11F4BAF
:10A580009B69E3402B4213D0E3B218000193FFF71D
:10A5900025FE01000198FFF755FFE3B2143B022BA3
:10A5A0001DD801217156184A8D405369AB43536140
:10A5B0003B7F002B0DD0E5B22800FFF795FF280068
:10A5C000FFF70CFE7B7F0100834202D02800FFF7DB
:10A5D000A5FD01340C370236172CC3D1F7BD01217C
:10A5E00000237156F3568D40074A9B009B189A68CA
:10A5F000AA439A60DCE7C04600E100E0FC65FF1F6B
:10A6000075BE0011FD65FF1F00F0004070B50E0023
:10A6100015000400FFF72AFF0C236343094A2000BA
:10A620009B189D605E60FFF75FFFF021064B074AB5
:10A630008900051E5A5002D02000FFF717FF28009E
:10A6400070BDC0461866FF1F0000FF1F79A10011F2
:10A6500070B5134D07202C78002C1FD198222100B3
:10A660005200280001F064FA0123C420FF222B705D
:10A670000C4B80001C635C630B4B1C605C600B4BE1
:10A68000195891433F3A0A431A50802252021A60E5
:10A690000D20074A074901F0DBF8200070BDC046D5
:10A6A000FC65FF1F00800040A0F0004000E100E0DA
:10A6B00045A5001145A30011030010B50620072B86
:10A6C00009D8054A137001F09BFAD7210020034BEB
:10A6D000034A89005A5010BD4843FF1F0000FF1F66
:10A6E000911BFF1F70B51D0002240C2910D8094AC8
:10A6F000CA40D2070CD5FBF741FF041E08D1059ACA
:10A7000004992800FBF756FFFCF7C4FDFFF724FB74
:10A71000200070BD1210000030B50D7802232C000F
:10A720009C43184201D02B431C0008252300AB4357
:10A73000284201D02B00234320241D00A5432042A2
:10A7400001D01C4325002A230D70184204D0117833
:10A750001E3B0B43137030BD0028FCD10C21137835
:10A760008B43F7E7F8B51D0006AB1B88140007AA5A
:10A770000E000B201778002B27D10A78022A49D126
:10A780004A68507811780002244A08438018042847
:10A7900040D801F0F5F903121D1B2300F06801F009
:10A7A000F7F8021CC0B2B84200D93A1CD2B220005D
:10A7B000F1682A8000F024FF06E00222F3681B887B
:10A7C0002A8023701B0A63700020F8BD0622EEE782
:10A7D00001232B80F3681B782370F5E7F368002BC7
:10A7E00016D008222A801A8822701A88120A6270EB
:10A7F0005A88A2705A88120AE2709A8822719A883E
:10A80000120A6271DA88A271DB881B0AE371DBE746
:10A810002B80D9E701202B80D7E7C04600D6FFFF69
:10A82000F7B516000A781D0008AB1F880C0001233D
:10A83000022A18D14A685078117800022B4A08433E
:10A84000801803280FD801F09BF902254439E068ED
:10A8500001F09EF8C0B20723B84204D37B190193DC
:10A86000152B02DD0D231800FEBDE0682A00310023
:10A87000C01900F0C5FE6B4600209B88E268D054EA
:10A880001B4B1B68834203D01B68834200D0984750
:10A890000023E8E70B23002FE5D1022DE2D17378E6
:10A8A00032781B021343E2681380114B1B68002BA4
:10A8B000EED01B68002BEBD00120E8E70B23002F24
:10A8C000D1D1062DCED12A003100E06800F098FEEB
:10A8D000DEE70B23002FC6D1012DC3D132787533AB
:10A8E000012AC0D8E3681A70D2E7C04600D6FFFF3D
:10A8F0000868FF1F70B50C001500072837D801F055
:10A900003FF9041436361B36242E182015290BD88F
:10A91000184E16220021300000F0A2FE220029006D
:10A92000300000F06DFE002070BD18200229FBD120
:10A930001288114B1A80F6E718200829F4D10A0072
:10A940000E48290001F09CF8EDE718200129EBD111
:10A950000B4B10780B49DA69FFF7DEFEE3E71820AE
:10A960000129E1D1064B10780749DA6BF4E70220A0
:10A97000DAE7C046F067FF1FC643FF1FBC43FF1F57
:10A980004C43FF1F7443FF1F9443FF1F030010B588
:10A990000020DB0704D50721024A034800F08CF8A9
:10A9A00010BDC04600BF00114C43FF1F054A030005
:10A9B0001068002803D082889A4201D180687047CD
:10A9C0000068F6E7006AFF1F0A88030008009A4241
:10A9D00004D08A8804309A4200D0002070470000DA
:10A9E000F8B5F22200230D4F0D4E79680500424361
:10A9F0003370994200D07B600A4C0021200000F0A7
:10AA00002FFE00231A007C60AB4202D1002033707D
:10AA1000F8BD01332280DBB2F234F5E7F86AFF1F9C
:10AA2000F66AFF1F046AFF1F73B56B4601900600AC
:10AA3000684615001980FCF75FFF041E11D1002D38
:10AA40000FD07689002E11D00C2000F031FE0028A6
:10AA50000ED0084A0460136886808560002B02D1FE
:10AA60001060200076BD1A001B68F7E70224F8E7A3
:10AA70001324F6E7006AFF1F012100220A4B10B5DC
:10AA800049420A4C198099809A719A70084B20703B
:10AA9000012019805A60FFF7A3FF2078FCF78AFF96
:10AAA0000448FDF745FF10BD1068FF1F006BFF1F36
:10AAB000F86AFF1F65AB0011022310B5002802D011
:10AAC000FFF7B2FF0300180010BD0000030010B52F
:10AAD0000020DB0704D50421024A0348FFF7A4FF46
:10AAE00010BDC04614BF0011CC43FF1FF0B50E26A9
:10AAF00087B003930CAB1F8802ABF6180500080063
:10AB000031000292FDF77AF804000120002C0FD0EA
:10AB10003088FFF74BFF03000E20002B08D05E6843
:10AB2000002E05D021002800039B029A0097B04711
:10AB300007B0F0BD0A4B10B5984207D1012200239F
:10AB400052420A808B708A808B7110BDFFF73CFFE8
:10AB50000028FAD001235B42038000238370F4E7CE
:10AB6000FFFF0000F8B5050001290AD1134E0024AB
:10AB70003388F227AB4219D028001149FFF7DAFFDA
:10AB800006E0022904D10139FDF750FF0028EDD07D
:10AB9000F8BD3B0063437268D018D35A002B09D02C
:10ABA0003A00002100F05CFD0134E4B2054B1B7853
:10ABB000A342EED801235B423380DDE7F86AFF1F32
:10ABC0001068FF1FF66AFF1F10B5FFF7FDFE0300B8
:10ABD0000020834200D0987810BD0000F0B589B005
:10ABE0001C000EAB80CB03901E8810AB1B78049228
:10ABF00002930B7A0D00DB0616D42B780593022BFB
:10AC000024D00498FFF7D2FE002812D003689C4697
:10AC1000002B0ED0029B2200019329003B006446CA
:10AC200003980096A04705E00498FFF7BFFE0028B0
:10AC300002D10E2009B0F0BD8368002BF9D00A22A2
:10AC40002900039898470028D7D0F3E76B68587815
:10AC50001A786B4B000210439842D2D8043B9842BA
:10AC600010D2684B984242D015D8674BC0180128C3
:10AC7000C7D80B20002EDDD1EB681A7859683A80CE
:10AC8000200028E0614BC018032800D979E000F0CB
:10AC900077FF846A789E5E4B9842B2D10B20002EDB
:10ACA000C8D101233B80EB6831001B782370688991
:10ACB000013080B2FCF7A2FF3A88031E0ED0017863
:10ACC00002328A183A80428962704289120AA2705E
:10ACD00059680278E01C00F093FC06E004323A80E8
:10ACE00031000422601C00F0BBFC0020A2E70B2016
:10ACF000002E9FD1EB6807A91E8804233B80330AEE
:10AD0000300026706370FCF779FF051E28D004AB75
:10AD10009A890E2304A95B183E49C668FCF7E2FF36
:10AD200000280BD12B783C486A680599FBF798FB03
:10AD3000002803D1012304AA5B42D3813278022A7E
:10AD400006D17168201D00F05BFC3B8802333B801C
:10AD50000E2304AA9B181B88A3701B0AE370C4E788
:10AD600004ABDE81F4E70B20002E00D062E7E96837
:10AD70000398FFF729FF02233B802070000A6070D0
:10AD8000B3E70B20002E00D054E70222EB681B88AB
:10AD90003A8023701B0A6370A7E7E86800F0F8FDAB
:10ADA000C2B203000720B24200D243E70DD002999D
:10ADB000DBB27118994202DB921BD3B20293029B61
:10ADC000E9681A003B8089195AE70023F6E70B204F
:10ADD000002E00D02EE70722EB683A801A78227006
:10ADE0005A7862705A88A2705A88120AE2701A79E8
:10ADF0002271DA886271DB881B0AA37175E7C0468D
:10AE0000042900000228000000D8FFFFFFD6FFFF42
:10AE100003280000FFFF000044BE0011F0B58DB014
:10AE20006B460020089120229B5E83423DDAA64BB0
:10AE3000187800F0EDFD071E32D00378B02B2CD12E
:10AE40000079023816281FD800F052FD17001E00A6
:10AE50001E001E0031001E0096001E001D011E0077
:10AE600052011E0073011E00CD011E0050021E0083
:10AE70001E001E008E021E00E302944B94491B88A4
:10AE800078880B80FBF72CF83800FCF7ADFF914B6E
:10AE90001B68002B01D038009847380000F0D0FB29
:10AEA0008020089B0002434018000DB0F0BDEE2248
:10AEB0000021874800F0D4FB0BAA3B7B79893889B5
:10AEC00000923A000D32FCF7B1FD0400804B1B7874
:10AED000002C3FD146E0804B788805937F4B4100A2
:10AEE000CB5A0BAE073BDBB23288029300230193AF
:10AEF0007B4B210006930093059BFFF76FFE744D7B
:10AF0000002810D1069B3A8A1B889A420BD1380040
:10AF10000599123000F0F4FD002804D02B786289E6
:10AF20009B00EB185A80162306A81B1832882000B5
:10AF30007989FCF7D7FE2B7804009A00AA1851886B
:10AF40000029C3D00133DBB22B70002807D006A93B
:10AF5000C98A9180634A12889A42BCD802E00121D2
:10AF600049429180002B04D059497888FAF7ECFFC8
:10AF70008AE73E890A2479E000253E89574B0693EB
:10AF80007B88069A5B009B5A033B9D4202DB002DA7
:10AF9000F0D05BE0162206A812183B7B798900925C
:10AFA0003A0030000D32FCF741FD0590002858D0E2
:10AFB0004689017A7888FCF703FD041E44D1464B8C
:10AFC00078880793069B4100C95A454B0439C9B29A
:10AFD00006AAD28A06930291019400930599079BD1
:10AFE000FFF7FCFD041E2FD1069B39491A88931CDC
:10AFF000002D26D14B807988384B4900CB5A511906
:10B00000033B8B4220DD059B31485B8941190B7165
:10B01000A91C0135C9B2EDB2059145191B0A2B7166
:10B02000059B2D490433181800F0EAFA2C4B059AB9
:10B030001B88D318DDB22C4B9E4205D00136B6B228
:10B040009CE749889942D6D0002D0CD0204C28008E
:10B05000618800F0B5FA207021007888FAF784FF43
:10B0600012E7059CF0E7002C00D183E77B78142BD6
:10B0700000D109E716493B794E800B700C71788836
:10B08000FAF724FF00E7162406ABE41821003889FC
:10B09000FCF7B4FD011E00D1B7E1788822880F4C7F
:10B0A00045002C5B0A4D013CE4B2029400240F4B96
:10B0B00001940095FFF792FD041E00D014E12900D1
:10B0C0007888FAF761FFDFE6006BFF1FB842FF1FC9
:10B0D0001868FF1F0C68FF1F0C69FF1F4864FF1FE3
:10B0E000FC69FF1FB642FF1FFFFF00001A68FF1F29
:10B0F000162406ABE41821003889FCF77FFD011EF9
:10B1000000D182E178882288AE4C45002C5BAE4DA0
:10B11000013CE4B202947C89AC4B01940095FFF7AA
:10B120005DFD041E00D0DFE029007888FAF736FFC5
:10B13000AAE60025A44B1D803B00F6331B78A24AEB
:10B1400078880792AB4208D99E4B128806930699DD
:10B1500043005B5A013B9A4203DB0799FAF728FF49
:10B1600092E616246B00FB18059306ABE418059BCA
:10B1700021001889FCF742FD011E03D1059B012423
:10B180001E8973E77888924B2288069C09934300B6
:10B190001B5B904E013BDBB20293002300960193B0
:10B1A000099BFFF71BFD041E02D0059B1E895DE76E
:10B1B0007B88069A5B009B5A079A1088328812187F
:10B1C000934202DC1B1A013B33807F4C02303288F1
:10B1D0000999001900F014FA2388328801359B1868
:10B1E0002380EDB2A8E70BAA3B7B798938890092CE
:10B1F0003A000D32FCF71AFC00250590059B002B48
:10B2000004D10A24002D00D16EE060E0059B78880F
:10B21000197AFCF7D5FB0100041E63D1694C6C4B15
:10B22000788806940993069B4400E45A694B063CCF
:10B23000E4B20BAE32880793029401910093059912
:10B24000099BFFF7CBFC041E4CD1079B5E491B8872
:10B250001A1D002D30D14A80059B5B4C5A89631919
:10B260001A716B1C9BB2E318120A1A71162306A8F6
:10B2700032881B1879890598FCF734FDFF21AA1C38
:10B280002E1D03350B00059092B2B6B2ADB2002868
:10B2900003D006ABDB8AD9B21B0AA218651911715B
:10B2A0002B714C4D301D2A884949201800F0A8F90F
:10B2B0002B88F618B5B2A1E74988914207D17A8860
:10B2C00006995200525AEB18053A9A42C4DC3E4C99
:10B2D0002800618800F0C4FA207021007888FAF70D
:10B2E00071FED1E5002DF2D13E89BFE6162606ABF0
:10B2F000F61831003889FCF781FC3D000400FA356E
:10B3000000282DD0037A9B060CD400227B89398932
:10B31000788800923A000C32FFF7E8FB041E10D048
:10B320003E8915E03088FFF741FB00281AD083687A
:10B33000002B17D02100122278889847041EE4D0F1
:10B34000EEE72B78002B02D17888FAF74BFE002627
:10B350002B78002B00D097E5002C00D194E585E6F2
:10B360000124DDE70E24DBE7162506ABED182900E6
:10B370003889FCF743FC041E47D0037A9B0611D49E
:10B38000154A7B881188994203D01448814207D11D
:10B390001380134BF2261D780023D9B2A94221D382
:10B3A0000924A1E72888FFF701FB00282FD0836834
:10B3B000002B2CD02100122278889847041EDFD061
:10B3C00092E7C0464864FF1F1868FF1F1A68FF1FF6
:10B3D0000C69FF1FFC69FF1FF86AFF1FFFFF0000D9
:10B3E000F66AFF1F31005943546801336018615AEF
:10B3F0000029D2D13C0008342100F22200F000F9EB
:10B4000021007888FAF7F6FD3EE501246CE70E246A
:10B410006AE71D4B1A887B889A4231D07888FAF700
:10B42000F3FD31E5F223059851684343CD18C95A1D
:10B4300000291FD03B7A012B0BD16C88AB88788810
:10B44000AA1D0094FFF752FB041E02D000233B729A
:10B450002E88F2220021280000F002F900232B8020
:10B46000059B0133DBB20593084B05991B78064A0F
:10B470008B42D7D801235B421380002CCED0F5E558
:10B48000002634000596EFE7F86AFF1FF66AFF1FF3
:10B4900070B504000E001500FFF796FA031E08D1E0
:10B4A00031000548FFF790FA03001120002B02D06D
:10B4B0001C8000209D7070BDFFFF0000F8B50B4F91
:10B4C00006003B780D001400FF2B0ED00A2000F080
:10B4D00067FB011E09D0B12303800023468003715E
:10B4E000C5800481387800F093FBF8BD0D44FF1F40
:10B4F000F7B50F0008A90600088809A90B240988D8
:10B50000002821D10234022B1ED1557813782D0248
:10B510001D432B008B4301937334002B14D1FB6824
:10B52000300019000093FFF74FFB019C85420BD0C0
:10B530002A0030000099FFF7ABFF041E04D12A0057
:10B5400030007989FFF7BAFF2000FEBDF0B50E7814
:10B5500085B003900AA805880120022E0DD14C6801
:10B560002778647824023C43054FBC4205D10398F8
:10B57000DBB201960095FFF7BBFF05B0F0BDC046FA
:10B5800002290000034B10B51B68002B00D0984720
:10B59000FEE7C046046BFF1F07B501A8FFF7F2FFE7
:10B5A000044A05480021121A00F0C2FAF8F722F9FD
:10B5B000FEE7C046086BFF1F1044FF1F000000009D
:10B5C00001B40248844601BC604700BF350E00004C
:10B5D00001B40248844601BC604700BFDD6601003B
:10B5E00001B40248844601BC604700BFE548000042
:10B5F00001B40248844601BC604700BF291C00001A
:10B6000001B40248844601BC604700BFE94C010018
:10B6100001B40248844601BC604700BF311B0000F2
:10B6200001B40248844601BC604700BF4550000099
:10B6300001B40248844601BC604700BF014C0100D0
:10B6400001B40248844601BC604700BF434D01007D
:10B6500001B40248844601BC604700BF4551010067
:10B6600001B40248844601BC604700BF154D01008B
:10B6700001B40248844601BC604700BFF13AFF1F95
:10B6800001B40248844601BC604700BF4D1F000062
:10B6900001B40248844601BC604700BF851F00001A
:10B6A00001B40248844601BC604700BF0919FF1F6E
:10B6B00001B40248844601BC604700BF3D4B010015
:10B6C00001B40248844601BC604700BFB14E00008F
:10B6D00001B40248844601BC604700BF8B520100A0
:10B6E00001B40248844601BC604700BF1D4B010005
:10B6F00001B40248844601BC604700BFB539FF1F52
:10B7000001B40248844601BC604700BF7136FF1F88
:10B7100001B40248844601BC604700BFE117000045
:10B7200001B40248844601BC604700BF156B0100AC
:10B7300001B40248844601BC604700BF25260000D2
:10B7400001B40248844601BC604700BFB54C01000B
:10B7500001B40248844601BC604700BFF94C0100B7
:10B7600001B40248844601BC604700BF6571010016
:10B7700001B40248844601BC604700BF017F00005D
:10B7800001B40248844601BC604700BFADAE000072
:10B7900001B40248844601BC604700BF3519FF1F51
:10B7A00001B40248844601BC604700BFD94901008A
:10B7B00001B40248844601BC604700BFE938FF1F5E
:10B7C00001B40248844601BC604700BF1147010034
:10B7D00001B40248844601BC604700BF5522000006
:10B7E00001B40248844601BC604700BFC9A90000FB
:10B7F00001B40248844601BC604700BF0D520100FD
:10B8000001B40248844601BC604700BF8D120000AD
:10B8100001B40248844601BC604700BFD91B000048
:10B8200001B40248844601BC604700BF5952010080
:10B8300001B40248844601BC604700BF8930FF1F45
:10B8400001B40248844601BC604700BF21460100A4
:10B8500001B40248844601BC604700BF1131FF1F9C
:10B8600001B40248844601BC604700BF090E0000D5
:10B8700001B40248844601BC604700BF0934FF1F81
:10B8800001B40248844601BC604700BF5147010033
:10B8900001B40248844601BC604700BFC56D010089
:10B8A00001B40248844601BC604700BF091B000088
:10B8B00001B40248844601BC604700BFC5210000B6
:10B8C00001B40248844601BC604700BFF537FF1F42
:10B8D00001B40248844601BC604700BF056A00000D
:10B8E00001B40248844601BC604700BFFD38FF1F19
:10B8F00001B40248844601BC604700BF353BFF1FCE
:10B9000001B40248844601BC604700BF75A900002D
:10B9100001B40248844601BC604700BFC92600004C
:10B9200001B40248844601BC604700BF791800009A
:10B9300001B40248844601BC604700BFEDA5000089
:10B9400001B40248844601BC604700BFC51D000029
:10B9500001B40248844601BC604700BF0D3BFF1F95
:10B9600001B40248844601BC604700BFE9280000DA
:10B9700001B40248844601BC604700BF4D36FF1F3A
:10B9800001B40248844601BC604700BF213AFF1F52
:10B9900001B40248844601BC604700BFDD5201008B
:10B9A00001B40248844601BC604700BF055E000048
:10B9B00001B40248844601BC604700BF3539FF1F0F
:10B9C00001B40248844601BC604700BF3D18000036
:10B9D00001B40248844601BC604700BF35550000F1
:10B9E00001B40248844601BC604700BF29510100F0
:10B9F00001B40248844601BC604700BFED4A010023
:10BA000001B40248844601BC604700BFC94A010036
:10BA100001B40248844601BC604700BFF54E0100F6
:10BA200001B40248844601BC604700BF4136FF1F95
:10BA300001B40248844601BC604700BF8552010042
:10BA400001B40248844601BC604700BFA54F010015
:10BA500001B40248844601BC604700BFA94601000A
:10BA600001B40248844601BC604700BF5125000074
:10BA700001B40248844601BC604700BF9DA9000094
:10BA800001B40248844601BC604700BF810E00003B
:10BA900001B40248844601BC604700BF456B010009
:10BAA00001B40248844601BC604700BF312EFF1F2D
:10BAB00001B40248844601BC604700BF4137FF1F04
:10BAC00001B40248844601BC604700BF7130FF1FCB
:10BAD00001B40248844601BC604700BF7539FF1FAE
:10BAE00001B40248844601BC604700BF350E000027
:10BAF00001B40248844601BC604700BFD932FF1F31
:10BB000001B40248844601BC604700BFCD4C01002F
:10BB100001B40248844601BC604700BF0124000014
:10BB200001B40248844601BC604700BF9D3AFF1F34
:10BB300001B40248844601BC604700BFB70E000054
:10BB400001B40248844601BC604700BF6DBC0000E0
:10BB500001B40248844601BC604700BF21240000B4
:10BB600001B40248844601BC604700BFC93AFF1FC8
:10BB700001B40248844601BC604700BF5D17000065
:10BB800001B40248844601BC604700BF213BFF1F4F
:10BB900001B40248844601BC604700BF691F000031
:10BBA00001B40248844601BC604700BF1D4D01003E
:10BBB00001B40248844601BC604700BF55490100FA
:10BBC00001B40248844601BC604700BFB352010083
:10BBD00001B40248844601BC604700BFF30E000078
:10BBE00001B40248844601BC604700BF090E000052
:10BBF00001B40248844601BC604700BFB132FF1F58
:10BC000001B40248844601BC604700BF911BFF1F7E
:10BC100001B40248844601BC604700BF594F01008F
:10BC200000030102020303030403050006020700E8
:10BC3000080209030A030B030C000D000E030F0397
:10BC4000100311031303140315021602A13B001184
:10BC5000D53B0011000000000200000062BC001192
:10BC6000192A0F180A000000F1590000FD240000F5
:10BC700041460100398000114DA00011A17400114E
:10BC80003D7E0011195300111DAE0011654F0011CA
:10BC9000B13D0011E13E0011000000001616000049
:10BCA00002000000ACBC0011F4FFF3FFD2FC000066
:10BCB000214000110000000000000000547579616F
:10BCC0000042312E340030303141006769746875AC
:10BCD000622E636F6D2F7076767800544842330081
:10BCE00002000000F4BC0011292A282A272A262A4B
:10BCF000252A242A0A180000E2040000710200002C
:10BD000078EC0000744000001027000060F0000094
:10BD100006640000204E0000000000000500000046
:10BD20001F501D00023CB40000011A001400000066
:10BD3000A1020000303132333435363738394142D0
:10BD400043444546000000001D5700117157001183
:10BD5000000000000200000060BD00116F2A6E2A82
:10BD60001A18EAD8BC80F0FC600000000000000057
:10BD700000005F066B2F363D7D077F3F777C596E55
:10BD80007971000001A00000000000006410B71DE0
:10BD9000C8206E3BAC30D9269041DC76F4516B6BF9
:10BDA0005861B24D3C7105502083B8ED44930FF0BB
:10BDB000E8A3D6D68CB361CBB0C2649BD4D2D38671
:10BDC00078E20AA01CF2BDBDFB349B5F80000080BE
:10BDD0000010000000000000A36000112D7700118A
:10BDE000C7600011357B00114B6100110B7B001106
:10BDF000C1610011E17A001113620011A97C0011E8
:10BE00007B620011A97C0011AD620011637C0011FE
:10BE1000C1610011997A001139620011417C001151
:10BE200000000000000000001F630011417C0011B1
:10BE30008163001145770011052A042A012A002A8E
:10BE4000022903280128002801180018000000001A
:10BE50000000000000000000000000870101020156
:10BE600002010102010203030401030101010101B6
:10BE70000303020103000D000E0010001100130067
:10BE80001401070108010A010B011C011D02040233
:10BE900005020702080219021A021C021D0301030F
:10BEA000020317000201000504000807000B0A0046
:10BEB0001716001D1C010201010504010E0D0111E0
:10BEC00010011413011716011A19020201020B0ABC
:10BED000020E0D02111002141302171603050403BB
:10BEE0000807030B0A030E0D0001020307090A0BE2
:10BEF0000E0F101112141718191A1B1F20212200DF
:10BF000065A7001121A80011000000000200000038
:10BF10004ABE0011000000004DB5001100000000F5
:08BF20000200000048BE001100
:020000041FFFDC
:1000000000000000193D001168BC001164BC001123
:100010004061FF1F00000000000000000000000021
:1000200000000000000000000000000000000000D0
:1000300000000000000000000000000000000000C0
:1000400000000000000000000000000000000000B0
:1000500000000000000000000000000000000000A0
:100060000000000000000000000000000000000090
:100070000000000000000000000000000000000080
:100080000000000000000000000000000000000070
:100090000000000000000000000000000000000060
:1000A0000000000000000000000000000000000050
:1000B0000000000000000000000000000000000040
:1000C0000000000000000000000000000000000030
:1000D0000000000000000000000000000000000020
:1000E0000000000000000000000000000000000010
:1000F0000000000000000000000000000000000000
:1001000000000000000000000000000000000000EF
:1001100000000000000000000000000000000000DF
:1001200000000000000000000000000000000000CF
:1001300000000000000000000000000000000000BF
:1001400000000000000000000000000000000000AF
:10015000000000000000000000000000000000009F
:10016000000000000000000000000000000000008F
:10017000000000000000000000000000000000007F
:10018000000000000000000000000000000000006F
:10019000FD32FF1F5D31FF1FC1660100000000003E
:1001A000000000000000000000000000000000004F
:1001B000000000000000000000000000000000003F
:1001C000000000000000000000000000000000002F
:1001D000000000000000000000000000000000001F
:1001E000000000000000000000000000000000000F
:1001F00000000000000000000000000000000000FF
:1002000000000000000000000000000000000000EE
:1002100000000000000000000000000000000000DE
:1002200000000000000000000000000000000000CE
:1002300000000000000000000000000000000000BE
:1002400000000000000000000000000000000000AE
:10025000000000000000000000000000000000009E
:10026000000000000000000000000000000000008E
:10027000000000000000000000000000000000007E
:10028000000000000000000000000000000000006E
:10029000000000000000000000000000000000005E
:1002A000000000000000000000000000000000004E
:1002B000000000000000000000000000000000003E
:1002C000000000000000000000000000000000002E
:1002D000000000000000000000000000000000001E
:1002E000000000000000000000000000000000000E
:1002F00000000000000000000000000000000000FE
:1003000000000000000000000000000000000000ED
:1003100000000000000000000000000000000000DD
:1003200000000000000000000000000000000000CD
:1003300000000000000000000000000000000000BD
:1003400000000000000000000000000000000000AD
:10035000000000000000000000000000000000009D
:10036000000000000000000000000000000000008D
:1003700099B500110000000000000000000000001E
:10038000000000000000000000000000000000006D
:10039000000000000000000000000000000000005D
:1003A000000000000000000000000000111BFF1F03
:1003B000000000000000000000000000000000003D
:1003C000000000000000000000000000000000002D
:1003D000000000000000000000000000000000001D
:1003E000000000000000000000000000000000000D
:1003F00000000000000000000000000000000000FD
:08183800106FFF1F4118FF1F94
:10184000024981F3088802F09FFB0000106FFF1F20
:1018500070B500241E491F4A1F484C6308CA1B0567
:101860001B0DE4188242F9D11C4B80228B630021AE
:1018700009201B4B920519621A4B1B4DDA671B4B53
:10188000DA688243DA609A68194802409A60112047
:10189000296002F08FF8112002F06CF86B6C154A89
:1018A000112013406B64EE23DB006343124A1B0CD0
:1018B00013840122114B9A7201F006FC104B1B7825
:1018C000002B04D10F4B1021187802F0C5F970BD20
:1018D000000005400806054080060540FF010000A5
:1018E00000F0004004E100E0003800403CF000401F
:1018F000FFDFFFFFFFFEFFFF1061FF1FC461FF1F3F
:10190000F263FF1FF061FF1F10B502F015FB0728FF
:1019100004D0122808D0022808D010BD044A0420A0
:10192000136B01331363F8E70220F6E71420F4E7A2
:10193000F064FF1FF8B507000C00260025005036A4
:1019400030785135002804D10300287058342370B2
:10195000F8BD2978CA00481E8141A3183800A25C4E
:101960005B68C9B2FFF7D0FF00280DD12B78DA00F1
:10197000A218013350602B703378044A013B337056
:10198000136A01331362D8E70123DFE7F064FF1F16
:101990005C234343074910B5C9180B0058331B7823
:1019A000012B05D1FFF7C6FF034A936A0133936207
:1019B00010BDC0462465FF1FF064FF1F10B502F084
:1019C000F3FA064A0121130010CB4942D967044BB0
:1019D000136002F0B1F9200010BDC04600E100E044
:1019E0001000100010B5040002F0DEFA024B1C607B
:1019F00002F0A2F910BDC04600E100E0431E5A42C9
:101A00005341A022F0B5D2015B421340154D164A56
:101A100040019B182A18127E8BB00191002A1BD01E
:101A20001A000832D46F0022E6B206AFE4B2944244
:101A30000EDC2818C369002B08D0019902AA117185
:101A400006AA049202AA167303A898470BB0F0BD29
:101A50001978B9540132EAE71A7D1A7806AB0126E3
:101A60001A70E6E7B067FF1F00400040F0B5254B55
:101A700004004001C25C85B0002A2BD01A18117EE8
:101A8000002927D0917E002924D01179022921D163
:101A90001689D788D168F51BADB22A1C102D00D944
:101AA000102292B2BE4217D11818012303710023ED
:101AB000C269C38003819A4206D06846032103733A
:101AC0000171029301A890470820002C00D0192032
:101AD00001F0FAFA05B0F0BD013C65426C41A02569
:101AE0006442ED012C40084D1B186419074D063364
:101AF000013A92B2AA42EDD01888461C1E80085CBA
:101B00002070F5E7B067FF1F00400040FFFF0000B6
:101B10000F220E4B10B59868104002380A280BD8D7
:101B200001F0FEFF0D0A0B0A0A110A0A0A0A060052
:101B300002210020FFF762FF10BD0121F9E700201C
:101B4000FFF794FFF8E7DB6FF6E7C0460040004080
:101B50000F220E4B10B59868104002380A280BD897
:101B600001F0DEFF0E0A0B0A0A120A0A0A0A060030
:101B700002210120FFF742FF10BD01210800F9E713
:101B80000120FFF773FFF7E7DB6FF5E700900040F8
:101B900013B5334C2378072B3DD8324B1A78324B90
:101BA000002A39D18022196852020A431A6025207E
:101BB00001F0C0FE20232D4A11680B4380211360E1
:101BC0006B460422C90508680733104228D08021DB
:101BD0000422C905C86810422ED080212020C905E2
:101BE000CA688243CA6014221A701A78002A2FD158
:101BF0008021C905C86820320243CA6014221A70C5
:101C00001A78002A28D11A4B1A7D22785A601D2290
:101C10001A705932DA6013BD1A6816490A40C5E7CE
:101C2000086802430A6014221A701A78002ACED07B
:101C30001A78013AD2B2F7E7C8680243CA601422A0
:101C40001A7019784A1ED2B21A700029F9D1C4E765
:101C50001A78013AD2B2C7E71A78013AD2B2CEE77F
:101C60004843FF1F1044FF1F3CF000404043FF1F4C
:101C700000200040FFFFFEFF564B70B51B68012B94
:101C800003D1554A936D0133936501F0F5FF534B32
:101C9000534A1860534B544C1A600123534A136043
:101CA000534A13602378002B06D00622514952482C
:101CB00002F00AF900232370504A514B10681B7838
:101CC000C1B2002B0ED14F4CC0B223785BB2002BB7
:101CD0004FDB237824785BB264B21B0424021B1907
:101CE0001B1813600B1C50294ED95023464A4749F4
:101CF0001078DBB2FF2202284BD10868444C454DD6
:101D0000267890432A78964254D9227824782E78DF
:101D1000023B5D10A31B6B435201D31A10335B11BE
:101D20001843086001F0D8FF031F012B45D83A4B38
:101D30001B78002B06D0394B1B78002B02D00020DB
:101D400002F0BAF8A122364B92009978354B4A43FB
:101D50001B689B18832292009B181B78033B012B66
:101D600003D8AF20400002F087F801222E4BDA8220
:101D700070BD237824785BB264B2FF33FF341B0458
:101D800024021B190138ABE7CAB2022AAED20223E1
:101D9000ACE70868254C264D267890432A78964271
:101DA00008D9227824782D78023B5B10641B6343AA
:101DB0005201B2E72378DBB2B2E70228D5D11D4B3E
:101DC0001B78013B022B03D91B4B1B78022BCCD178
:101DD0006C20C8E79809FF1FFC0FFF1F3C64FF1F22
:101DE000FF3F0000141003404064FF1F0C1003402D
:101DF00000100340D50BFF1F7211FF1FB4000340FA
:101E00008C09FF1F680AFF1F490AFF1F9400034047
:101E1000460AFF1F470AFF1FF908FF1F2209FF1F7D
:101E2000300DFF1F3409FF1FBC0BFF1F440AFF1FAB
:101E3000450AFF1F1C09FF1F2309FF1F10B501F0F2
:101E4000FBFE0022014B1A8010BDC0463A64FF1F02
:101E500010B501F051FFA121054A89009478054A87
:101E600061431268044B5218528C1A8010BDC04650
:101E7000300DFF1F3409FF1F3A64FF1F10B50D4BD3
:101E80000D4A9978A1239B004B431268D218531D29
:101E9000D97F0A4B1B88994209D2441C07D0C82815
:101EA00005D0D2695B1A5A43054B5343C01802F060
:101EB00093F810BD300DFF1F3409FF1F3A64FF1F58
:101EC0007102000070B5244D2B68002B28D001F062
:101ED00073FF2B68D8402B680400002B27D001F03B
:101EE0003BFE2B68D8401D4B1D4A9978A1239B00CF
:101EF0004B431268D118D25C91239B00002A20D05A
:101F0000CA580132CA50174B17491B6808688342E8
:101F100014D3D23B181A012A1AD0144B186070BD82
:101F200001F04AFF124B196801F056FED3E701F0A9
:101F300013FE0F4B196801F04FFED4E70D495B18F3
:101F4000E8E7CA500C4B1B68DB68E418201AE4E78A
:101F5000F530FF30E1E7C0461C08FF1F300DFF1FC2
:101F60003409FF1F9C09FF1F3C64FF1FA009FF1FCE
:101F70001808FF1F2DFF3F004464FF1F70B50400C9
:101F80000D00282916D10300A433C2881B889B1A90
:101F90000B4A9BB293420DD906006A3605223100E6
:101FA000653001F021FE002804D13100200002F04C
:101FB00023F870BD2900200001F06EFEF9E7C0464D
:101FC000FE7F0000F8B50500012001F045FF134C2D
:101FD000A36AA26A9342FBD1114E336001F0BCFEAA
:101FE0001049030008601048426894460F4A176879
:101FF0000022BC4501D24268BA1A0D48026032681C
:10200000AD18A422E562606A520302436262094A83
:102010001278002A01D00F3B0B60F8BD00F00040A1
:10202000340AFF1FE408FF1F28100040180AFF1F92
:102030001C0AFF1F1C09FF1F70B580241025E40532
:10204000A3682B43A36001F09FFEA368AB43A3608A
:1020500070BD0000F7B5160080221C001023D205C9
:102060000191916805000B43936000225A4BD730D1
:102070001A6001F051FE9D232A002F009B00EB58AF
:10208000CA3201210092FC37002B01D00021009AB6
:10209000386801F011FE2900009BCB311A784F4BB4
:1020A000D3351A604B780A781B0213438A781204DE
:1020B0001A43CB781B061343494A1BBA13604B796A
:1020C0000A791B0213438A7912041A43CB7931002F
:1020D0001B061343434A1BBA13606B782A781B0212
:1020E0001343AA7812041A43EB781B0613433E4AA3
:1020F0001BBA1360019A330213433C4A13603C4BF2
:1021000022001B1B9C4603293DDCB3089A001300E8
:102110005142B21A032A46D1354AE018511A827840
:102120004078120400020243E05C043302430A6078
:102130000022FF2B4BDDF0222E4B12011A600F22E2
:102140002D4B1A602D4A1368002BFCD00023224A25
:1021500027491360091B321D0B191B68043A180A22
:1021600023706070180C1B0EA070E3700434002AFA
:10217000F2DC802210213B68D20501333B6093687A
:102180008B439360F7BD6346D578981893782D06F6
:102190001B042B43157804392B43557804322D0248
:1021A0002B430360AFE7022A0AD1114AE05C511ABF
:1021B000E2185278120202430A6004339BB2B7E776
:1021C000012AB5D10A4A521AE15C1160F5E70849C3
:1021D00059180A600433ACE7000004403C00044096
:1021E0003800044034000440300004400C00044037
:1021F00000010440040004401000044014000440A6
:10220000F7B5150080221C001023D20500919168BB
:1022100007000B4393600023654AD730136001F039
:102220007BFD9D233E009B00F9583B00CA363200DF
:10223000FC33002900D07FE0586801F03DFD3900F3
:1022400032785C4BCB311A604B780A781B0213430F
:102250008A78AC4612041A43CB78281D1B06134318
:10226000554A1BBA13604B790A791B0213438A79CA
:1022700012041A43CB791B061343504A1BBA13604E
:102280004B7A0A7A1B0213438A7A12041A43CB7AD6
:1022900021001B0613434A4A1BBA1360009A2B0203
:1022A0001343484A13602200474B1B1B0093009BBB
:1022B000CE785B1801938B7836061B0433430E7877
:1022C000043833434E78043136023343019E336081
:1022D0000328ECDC0321A808431C9B002940800054
:1022E00003292BD13849E5185E18A9786D78E35C8D
:1022F00009042D02294319433160030008330021EA
:10230000FF2B2DDD314B324919600F21314B196004
:10231000012327490B60304B19680029FCD00621A6
:102320001B680B40042B20D080220020D20593682C
:102330000A318B439360FEBD01217DE7022908D15C
:1023400021495D18E1184978E35C090219432960C5
:10235000D3E70129D3D11C495918E35C0B60CCE7C2
:102360001948181801600433CAE7002310490B60AC
:102370006346002B0CDC3B00FC335A681021013211
:102380005A608022D205936801208B439360D2E784
:10239000009B9B181B68190A13705170190C1B0EB7
:1023A000D37004235B4291709C440432E0E7C04642
:1023B000000004403C000440380004403400044065
:1023C000300004400C0004400001044004000440BC
:1023D000080F0000100004401400044070B5061EF1
:1023E00019D002225A4B9B799343012B13D1594B9D
:1023F0001A78FF2A0FD15A78FF2A0CD19A78FF2A2F
:1024000009D1DA78FF2A06D11A79FF2A03D15B793C
:10241000FF2B00D199E0504B0C201A78012A08D0EC
:1024200000224E4D1A7029780B00093B042B01D86D
:10243000212070BD4B1F012BFAD9454CA37B042BE7
:1024400000D982E0A279032A00D97EE09A1ED2B296
:10245000012A02D860881F2877D9002E56D0012E75
:1024600073D1A0880128E3D0002907D1581E032882
:1024700003D801F055FB121715122E702978481E4B
:10248000032811D80025364B1D602823237501F041
:102490000BFDA84227D0A580CAE702212970EDE7ED
:1024A0000421FBE70321F9E707390129C0D82D49A9
:1024B0000968C96A8906BBD52B4908780028B7D1B5
:1024C000012A01D9002BB3D102230B708021274DA3
:1024D000263389012878237501F08EFB8021287826
:1024E000890101F0B9FB0123A380214B1B78002B4C
:1024F0000AD0FA2280211F4B92001B8809025A43FE
:102500001A4B187801F010FC002092E701F04CFD06
:102510002B78A680073B012B03D917482E7001F0BA
:10252000B3FC114B114C1A78002A06D080210022EE
:10253000207889011A7001F05FFB01F0FDFB80211A
:102540002078090201F058FBDEE7122071E7C0464F
:10255000A60BFF1F6B09FF1F1A09FF1F1C09FF1F96
:102560004809FF1F4464FF1F2309FF1F1B09FF1FAA
:102570002109FF1F2C09FF1F0010004010B5002982
:1025800001D001F041FB10BDF7B5604B0191997886
:10259000A1239B004B435E4A060014681022E418F6
:1025A000D6235B00E0583623FF33E35C00279343D8
:1025B000222B41D1574B0F3A1A600760012501F0D9
:1025C000A3FC019B1880E8235B00E35C002B01D097
:1025D000B34258DD0023504FFB70AD33FF33E35857
:1025E0001A68002A03D09B88DB439B071DD0382341
:1025F000FF33E35C002B18D09B235B00E35C002BD4
:1026000013D1D133FF33E35CB3420EDAA4235B0072
:10261000E15AE018090A023101F026FC23000122E8
:10262000FE33013E01351A87FA70E8235B00E35C54
:10263000002B2AD0A8B2FEBD03683D00002BBED0FF
:1026400081880430090A023101F00EFCD6235B00B8
:10265000E3581F60B2E72300B133BA00FF33985844
:10266000013781880430090A023101F0FDFBE823BB
:102670005B00E35CBB42EEDCE822F61AED180023B7
:102680005200A354A6E70027F1E7200001F00CFB5D
:1026900000281FD0002E1DDD7319882647190193CD
:1026A000B600200001F078FC5A3080002018406805
:1026B000013581880430090A023101F0D5FB200080
:1026C00001F00AFCA3590133A351BD4202D0019B82
:1026D0009D42E6D1114BE35C002BABD095239B00D0
:1026E000E35C002BA6D00E4BE15A0029A2D00D4A84
:1026F000A35C994202D90133A3549BE700231A211A
:102700002000A35401F010FC94E7C046300DFF1FD9
:102710003409FF1F00140340E010FF1F5A0200009D
:10272000720200005E0200000D4970B54A6E0D4C49
:10273000D2038B69D20BA24206D80B4D0224AA42C7
:1027400004D901F051FB70BD02246442E218150067
:102750007E2425402242F4D0A3432B438B61F0E733
:1027600000F000400A200000FC1C0000F8B51D4BE2
:102770001D4F1A78002A10D1BA7B002A02D10132EB
:102780001A7003E0032AFAD0022AF8D001F08CFB79
:1027900000220120154B1A70F8BD154B154D1C6811
:1027A000154B9E7801232B702878C0B200F09EFB59
:1027B000BB7B002B0BD101F0C7FAA1239B00734315
:1027C000E41883239B00E41823782B70E4E7032BA1
:1027D00002D101F029FBF0E70020022BDCD101F04F
:1027E00023FCEAE71C09FF1FA60BFF1F2309FF1F9D
:1027F0003409FF1F490AFF1F300DFF1FF0B587B0D6
:102800000EAD2F780FAD2D780593AC4663461400BE
:102810000E4D0CAA12782E7803930D9B0092019313
:102820002200059B029701F0CFFA2E70012C01D0F7
:10283000042C08D1802206498B889343054A1278DC
:10284000D20113438B8007B0F0BDC0461C09FF1FA7
:102850006C11FF1F7809FF1F0B001B3B70B50400B4
:102860003020E02B0DD81300E025493BFF3B9BB205
:10287000ED00AB4205D8034B200019825A8201F0CB
:10288000E3F970BD8410FF1F10B501F0F5F9054B99
:1028900000205B68052B04D9034A5268D20200D499
:1028A000980810BD00100040FCE100E070B501F098
:1028B0007BFB0D4B1B68FC33DC691D6AFFF7E4FFF3
:1028C0006419844204D2094B01241B68002B07D0F1
:1028D00004220024064B1A70064A9369013393615F
:1028E00001F02AFA200070BD4464FF1F9809FF1F01
:1028F0002309FF1FFC0FFF1F70B50C4D2B68FC3325
:102900005C6A01F051FBFFF7BFFF2B680025FC3329
:102910009B6AE318834204D2054B1B68AB4200D18B
:10292000051B01F009FA280070BDC0464464FF1F72
:102930009809FF1FD722044B92009B5810B5002B1B
:1029400000D0984710BDC0460000FF1F10B501F031
:10295000CFF8FFF7EFFF2749274BCA6D274C1A40E6
:1029600084235B001343CB65254B1B68186A01F079
:1029700073FA244B244A1A60244B254A1A60A02279
:10298000244B52001A60244B187801F03DFA2000C5
:10299000224901F0D9FA0023A3600233A360204B3F
:1029A0002049236003232048A36001F0CDFA1022C0
:1029B0001E4BFF201A60802252031A60802292036D
:1029C0001A60802212041A6001F076FA012001F0E8
:1029D000CBFAFA20400001F0F7FA582001F04CFA47
:1029E000134801F0F9F9012001F0B6FA072001F0CF
:1029F0007BFA10BD00F0004000FEFEFF1410004006
:102A00004464FF1F000003400180063DBC000340FA
:102A100034080000A40003404A0AFF1F71020000AE
:102A2000C3090000FFFF3F002810004000E100E064
:102A300030750000674E336888331B6883F308885D
:102A400001F0E2FA644A6549136800200B40136004
:102A5000634B644A1B68934200D1A6E001F0C4FABC
:102A60000221614A13688B431360FFF76FFF5F4BCE
:102A70005F4C1878C0B201F08FF80023A3600233D6
:102A8000A3605C4B0120236001F0E6F90323A360FF
:102A900001F0CAF8040001F0EFF8050001F0C4F8F5
:102AA000554B186001F080F9544B1968621A531E97
:102AB000A14200D213008022D203934201D39B0291
:102AC0009B0A3268D16AC90700D471E04C491C0CDA
:102AD00009689BB24C4359432402090A641803262F
:102AE0004849FC3293680A6847489B1A474A076876
:102AF000126847499B18474A9A1833409208DB19D5
:102B00000A600360042B03D9013233400A6003607A
:102B10000E684149A619300001F05EF83F4F3E496A
:102B20003B68C3183B603000019301F085FA3C4ECE
:102B30003068081838493060884205D9019B013354
:102B40003B6001F079FA316001F016F9354B1B78E2
:102B5000002B0DD001F090F8334B621B196812184E
:102B60008A4232D24919091B091A304801F0ECF99E
:102B70002F4E337A002B0ED001F07EF8621BF168E5
:102B80001218914224D94919091B091A294801F040
:102B9000DBF900233372284B83F3088800F0E4FF4D
:102BA000002001F021FA01F06FF801F01DFA5CE756
:102BB000DC0199000234641A5900641A09214B435C
:102BC0008033CB40A408E41889E7FA218900CCE7D8
:102BD0001A49DBE74464FF1F1CF00040FFFFC1FF00
:102BE0000C0AFF1FB641210310000040490AFF1FD5
:102BF00014100040C3090000100AFF1F340AFF1F11
:102C0000380AFF1F200AFF1F280AFF1F1C0AFF1F88
:102C1000240AFF1FC4090000710200006008FF1FA2
:102C20002C0AFF1F1C09FF1FE408FF1F00100040B3
:102C3000740BFF1F3C10004000000020DC0500006A
:102C4000A022054B92009B5810B5002B01D098474D
:102C500010BD01F021F9FBE70000FF1FA122054B89
:102C600092009B5810B5002B01D0984710BD01F081
:102C700013F9FBE70000FF1FA222054B92009B58AF
:102C800010B5002B01D0984710BD01F005F9FBE706
:102C90000000FF1FA322054B92009B5810B5002B8C
:102CA00001D0984710BD01F0F7F8FBE70000FF1FC7
:102CB000A422054B92009B5810B5002B01D09847D9
:102CC00010BD01F0E9F8FBE70000FF1F70B500F050
:102CD000D3FF4F4B186000F077FF0400C30702D406
:102CE00000F062FF70BD00224A4B1A604A4B187810
:102CF0000138042829D800F013FF0320181C2400F1
:102D0000200000F0B1FF0128ECD0444C2378042BC4
:102D10006ED100F051FF0028E4D000F07DFF582074
:102D200001F0AAF802232370DCE7200001F074F917
:102D3000E9E7200001F060F8E5E7200001F03CF948
:102D4000E1E7200001F018F9DDE700F0C5FF05001C
:102D5000012808D1324B1B78053B012B03D82000FA
:102D6000FFF76EFFD1E72D4B1B78022B01D0052B0F
:102D700020D1022D28D12B4B9B7BAB431CD12000B3
:102D8000FFF76CFF264B18780128BED16405BCD430
:102D9000244925224B7B034205D1233A13405A4252
:102DA000534126331A000B7D9342AED9322000F0F6
:102DB000DBFFAAE7022D07D1194B1B78052B11D198
:102DC0002000FFF759FFDDE7012D0BD1012B03D1C7
:102DD0002000FFF75FFF98E7062B03D12000FFF7E5
:102DE00067FF92E7200001F057F8022D8DD1C9E767
:102DF000032B04D10C4B987C00F086FF72E7072B65
:102E000000D06FE7094B987B00F0B6FE6AE7C0463A
:102E10009C09FF1F9809FF1F9009FF1F2309FF1F2F
:102E20001C09FF1FA60BFF1FBC0BFF1FD40BFF1FAE
:102E3000FA210A4B0A4A49001A640A4A5A500A4AB5
:102E400004395A50094A08319A64094A5A50094AC1
:102E50005C315A50084ADA667047C0460000FF1FCE
:102E6000FD27FF1FF928FF1FAD28FF1FDD23FF1FD0
:102E70006D27FF1F7D1EFF1F511EFF1FF7B50B0C97
:102E8000FF270122009300233C001E001D009446F2
:102E9000019089B262469A401000084018413618E5
:102EA000B6B2FF2F02D1012E00D19FB2009802408E
:102EB0001A41AD18ADB2FF2C02D1012D00D19CB248
:102EC0000133102BE6D10320012E07D1012D04D1AF
:102ED000019B2401E4191C700138FEBD102EFCD1A9
:102EE0000238102DF9D00230F7E700008023F7B543
:102EF0009C46264B264F01932649274A274D284CAE
:102F0000284B02281AD1604638600868264E3040A7
:102F1000802636033043086001990978002909D1D9
:102F20001660224A2A60224A2260E02219689143F0
:102F3000A03A1BE08021C9021160F2E766463E60BC
:102F40000F68194E3E408027FF023E430E600199F4
:102F5000097800290DD1176001280ED1154A2A6081
:102F6000154A2260E02219689143C03A0A431A6068
:102F7000F7BD802189021160EEE7E0210F4A02438C
:102F80002A600F4A22601A688A43F0E74B0AFF1F43
:102F9000E0000340D80003409000034000000340DD
:102FA0005000034040000340FFFFE3FF0280063D66
:102FB000804508220180063D806608220080069830
:102FC00080550822F8B51E4B80261A680020140090
:102FD0003440324232D11A681A4F32431A60012209
:102FE0003B68063093433B6000F036FF0122164DEC
:102FF0002B681E432E603B680A2613433B608027E4
:10300000BF00124B1B683B4211D1013EF6B2FF2EAE
:1030100009D17E220E4B1C682B68E40B14409343AD
:1030200023432B6005E0082000F016FFE9E7002E9F
:10303000EFD180222B68600893432B60F8BDC04617
:10304000C4F000405CF0004018F0004068F0004020
:1030500060F0004010B500F05FFF01215820034AE6
:1030600000F042FEFFF7AEFF10BDC046600AFF1F32
:1030700010B578220021034800F0CEFE00F064FD78
:10308000002010BD3867FF1F70B5040000F08CFFF2
:1030900000230C200B4A010059438D18515C002974
:1030A0000DD0A14208D1012300246B7000F024FF51
:1030B00000F042FE200070BD01330A2BEBD1122438
:1030C000F6E7C0463867FF1F70B5040000F06CFFDC
:1030D000002319001D000D4A1078002806D0A042D8
:1030E0000CD1557001310C320A29F5D1002B0AD1CF
:1030F00000F02AFD00F020FE002070BD5078461E32
:10310000B0411B18EEE700F0F7FEF3E73867FF1F4A
:10311000F7B504000C20002384460E4D019267464B
:103120005F43E85D7E19A04212D000280BD10A4B04
:103130009C4662461B7808331370019B70707C5567
:103140007160B360FEBD01330A2BE8D10320F9E7BB
:103150000720F7E73867FF1F3467FF1F8020F8B5A7
:10316000484BC0051B68C1248360474BFF251A6884
:10317000012313434361454BA4001A68444B40218B
:103180001A60444B1A68444B1A60444B1A59AA43BC
:103190001A51C52292009E58AE4331438026995061
:1031A0009F583F49F6010F403E439E509E5880274E
:1031B0003602360A3043985080201A5900020A40DD
:1031C00002431A5104341A59364E3F0432408026C5
:1031D0003A431A511A5936061202120A32431A5148
:1031E00008341A5980260A4002431A51C322920019
:1031F0009F58B446AF4337439F509F58294E0F40C6
:1032000007439F509F583740802636043743802617
:103210009F509F5836063F023F0A37439F50C022B7
:103220001F59AF433A431A511A591202120A164350
:10323000C6221E5192009C58AC4365462C439C50BC
:103240009C5800250C4020439850C72080001A58F5
:10325000154C1140C02212020A431A50134B1B781E
:10326000DB08AB4201DC0020F8BD2378002B06D040
:10327000A368002B00D0984701350C34EEE71220EC
:10328000F2E7C0464443FF1F4043FF1FB0F0004039
:103290003067FF1FB4F000402C67FF1F00E100E023
:1032A000FF00FFFFFFFF00FF3867FF1F3467FF1FAE
:1032B000030010B51F2809D8072200201340072457
:1032C00004490A78A24313430B7010BD0023062063
:1032D000F5E7C0463467FF1F054B06491B780A68AF
:1032E00005485B0702401B0B134300200B6070472F
:1032F0003467FF1F1CF00040FFFFC1FF70B50C25B5
:10330000FFF7EAFF0A4B1C780A4BE4086543ED1807
:10331000002C01D1200070BD2B78002B06D06B68EB
:10332000002B00D09847013C0C3DF1E71220F2E75A
:103330003467FF1F2C67FF1F1FB5002102220B00FF
:1033400001910091052000F01FFC02230B490A683F
:103350001A42FCD120230393039B5A1E0392002B95
:10336000FAD1074A1368002BFCDA0B246C442000C6
:10337000012100F069FD207804B010BD90C8004024
:1033800000C8004013B504000A4B0193019B002BB9
:1033900001D1112016BDFFF7CFFF230003400442E7
:1033A00005D0052000F058FD019B013BEDE718001A
:1033B000F0E7C046FFFFFF0707B500F0F5FD8022EC
:1033C0000821D205936A0191002B01D1073991623E
:1033D00002210C4A11600199481E01900029FAD17E
:1033E00003311160053101910199481E01900029B6
:1033F000FAD11160002B02D18022D205936200F035
:103400009BFC07BD00C00040F0B52D4C89B023786F
:10341000002B4FD1FEF7D2FA02232A4F03903A68CD
:103420001A42FCD120230693069B5A1E0692002BBB
:10343000FAD1254E3368002BFCDA0120FFF7A2FFFA
:10344000011E02D0112009B0F0BD0300032201903B
:10345000009005AD9F2000F097FB0321280000F0AD
:10346000F3FC02233A681A42FCD120230793079BFE
:103470005A1E0792002BFAD13368002BFCDA012088
:10348000FFF780FF0028DDD10398FEF7ABFAAA789A
:103490006B7811041B020B4329780B436360130004
:1034A000113B0A49052B07D801239340A3600B6009
:1034B000012323700020C6E780231B03F6E7C046E4
:1034C0002C43FF1F90C8004000C800409808FF1F11
:1034D0001E4B30B55A6818781D4B85B0D318594229
:1034E0004B4101210093002300F0EEFB194B1A4AD7
:1034F00002259A6300221A6510325A658022C4217F
:103500009D65164B1648D202DA6789004258154B62
:1035100080241A4080231B0413434350642341201A
:103520000393E40500F006FA402000F003FA656218
:10353000039D6B1E0393002DFAD103236362FFF7F3
:103540003BFFA562FFF760FF05B030BD3843FF1FAA
:1035500095FFFEF700C80040050001FF04E100E010
:1035600000E100E0FFFF00FFF0B585B00700FEF7C7
:1035700025FA022305002D4C22681A42FCD1202393
:103580000093009B5A1E0092002BFAD1284E3368FC
:10359000002BFCDA0120FFF7F5FE002803D01124F0
:1035A000200005B0F0BD234B2360022322681A429D
:1035B000FCD120230193019B5A1E0192002BFAD1CA
:1035C0003368002BFCDA0120FFF7DCFE0028E6D18F
:1035D000194B1F60022322681A42FCD12023029358
:1035E000029B5A1E0292002BFAD13368002BFCDAA0
:1035F0000120FFF7C7FE0028D1D1104B2360022322
:1036000022681A42FCD120230393039B5A1E039283
:10361000002BFAD13368002BFCDA0120FFF7B2FE51
:10362000041EBCD12800FEF7DDF9B9E790C80040C0
:1036300000C8004001000006A8C800400180000149
:1036400010B50020FFF790FF10BD000010B5064B2D
:1036500018705960FFF73CFF00211320034AFFF761
:1036600057FD002010BDC0463843FF1FD134FF1F57
:10367000F0B5040085B003920291FEF79FF988220D
:1036800063035B0B52051A438023DB059D6A80238D
:10369000274F0092BA68002601901B039A420CD96A
:1036A000F82326001B041E401C4206D08022214B1A
:1036B00052025E6219680A431A60002D0BD100F0B5
:1036C00073FC02221C4B1A608023DB055A62013A0C
:1036D0009A6200F031FB0023039A934220D1002D1F
:1036E0000AD100F061FC144B03221D608023DB052E
:1036F0005A629D6200F020FB8023BA681B039A4245
:1037000008D9002E06D000220A4B0C495A621A68CA
:103710000A401A600198FEF765F9002005B0F0BD77
:10372000009A0299D2181278CA540133D4E7C046DD
:103730002C43FF1F00C8004000C00040FFFFFEFFF9
:10374000F0B587B0029103920400FEF737F90190BB
:1037500000F02AFC802302250122234EDB05356080
:103760005D629A6200F0E8FA204F3B682B42FCD180
:1037700020230493049B5A1E0492002BFAD11C4D63
:103780002B68002BFCDA0120FFF7FCFD002802D09B
:10379000112007B0F0BD2000039A029900F0FCFA56
:1037A000022304003A681A42FCD120230593059BAA
:1037B0005A1E0592002BFAD12B68002BFCDA01204F
:1037C000FFF7E0FD051EE3D100F0EEFB80230322AE
:1037D000DB0535605A629D6200F0AEFA0198FEF793
:1037E00001F9E0B2D5E7C04600C0004090C80040F3
:1037F00000C80040F0B5802489B00600FEF7DEF86E
:10380000E405A36A02250393029000F0CDFB012397
:10381000304F3D606562A36200F08EFA2E4C236843
:103820002B42FCD120230593059B5A1E0592002BA9
:10383000FAD12A4D2B68002BFCDA0120FFF7A2FDFC
:10384000002803D01124200009B0F0BD244B2360D0
:10385000022322681A42FCD120230693069B5A1E9B
:103860000692002BFAD12B68002BFCDA0120FFF71F
:1038700089FD021EE6D11B4B03211E60030001904F
:103880000090202000F080F9022322681A42FCD127
:1038900020230793079B5A1E0792002BFAD12B680F
:1038A000002BFCDA0320FFF76DFD041ECAD100F0E7
:1038B0007BFB80230322DB053C605A629C6200F0A4
:1038C0003BFA039B002B01D1FFF776FD0298FEF730
:1038D00089F8B8E700C0004090C8004000C8004028
:1038E0000100000694C8004007B5000201910422BF
:1038F000000A01A9FFF724FF0EBD000073B5050003
:1039000005240B4AA3005B429B1819686B46DE1D19
:103910003000FFF7B3FA022804D133782B55013C6D
:10392000EFD276BD052CFCD00128FAD10230F8E7A1
:10393000140900111F2807D8012380228340D205D3
:1039400091680B43936070473F2808D80123802279
:1039500020388340D20551690B435361F3E75F2858
:10396000F1D80123802240388340D205116A0B43ED
:103970001362E8E71F2807D8012280218240C90589
:103980008B6893438B6070473F2808D801228021C1
:1039900020388240C9054B6993434B61F3E75F28A8
:1039A000F1D80122802140388240C9050B6A934337
:1039B0000B62E8E71F2810D880230200DB05153AC8
:1039C0001968012A06D820229143196019680A4310
:1039D0001A60704701228240F6E73F2811D8802301
:1039E0000200DB05353AD968032A06D81022914334
:1039F000D960D9680A43DA60EBE7012220388240B7
:103A0000F5E75F28E5D842238022181A413B83401E
:103A1000D205516A99435162516A0B435362D8E708
:103A200010B50400012813D1A022184992050B6893
:103A30005B015B0913430B60154B164A1968114073
:103A4000154A0A431A60402219680A431A6010BDD9
:103A50000028FCD101000A2000F0EEF921000B2023
:103A600000F0EAF9C0220A4B920019680A4340218B
:103A70001A601A688A431A60B022044912060B6859
:103A80005B015B0913430B60E1E7C04614F00040A3
:103A90001CF000407F00FEFF80FD010072B6074A67
:103AA0001368013313600422054B1A600023054A92
:103AB00013608022D2055360FEE7C0467808FF1FDE
:103AC000C0F00040C4F0004005490B68002B05D150
:103AD000044A0A6004490A60044A13607047C046F9
:103AE000140AFF1F841E0000380AFF1FC4F00040A4
:103AF0000023034A1360034A1360034A13607047AC
:103B000054F0004040F1004044F1004002B47146DE
:103B100049084900095649008E4402BC7047C04616
:103B200002B4714649084900095C49008E4402BC50
:103B30007047C04603B47146490840004900095A1D
:103B400049008E4403BC704701B40248844601BC5E
:103B5000604700BFADAE000001B40248844601BC1E
:103B6000604700BF6D0B010001B40248844601BCF0
:103B7000604700BF7997000001B40248844601BC49
:103B8000604700BFC1F7000001B40248844601BC91
:103B9000604700BF496D010001B40248844601BC82
:103BA000604700BF8914010001B40248844601BC8B
:103BB000604700BFDD0A010001B40248844601BC31
:103BC000604700BF01D7000001B40248844601BC31
:103BD000604700BFBD0B010001B40248844601BC30
:103BE000604700BF090E000001B40248844601BCD2
:103BF000604700BFCD4C010001B40248844601BCBF
:103C0000604700BFB352010001B40248844601BCC2
:103C1000604700BFE9D4000001B40248844601BCFB
:103C2000604700BF6DF6000001B40248844601BC45
:103C3000604700BF156B010001B40248844601BC17
:103C4000604700BF8D82000001B40248844601BC79
:103C5000604700BF116E000001B40248844601BCF9
:103C6000604700BF0D52010001B40248844601BC08
:103C7000604700BF0134010001B40248844601BC22
:103C8000604700BFC95C010001B40248844601BC22
:103C9000604700BF8552010001B40248844601BC60
:103CA000604700BF51B8000001B40248844601BC1F
:103CB000604700BF71B0000001B40248844601BCF7
:103CC000604700BF2144000001B40248844601BCA3
:103CD000604700BFC56D010001B40248844601BCC5
:103CE000604700BFDD0C010001B40248844601BCFE
:103CF000604700BF0167010001B40248844601BC6F
:103D0000604700BFF9ED000001B40248844601BCE1
:103D1000604700BF4DF9000001B40248844601BC71
:103D2000604700BF8944000001B40248844601BCDA
:103D3000604700BF8B52010001B40248844601BCB9
:103D4000604700BF9DA9000001B40248844601BC41
:103D5000604700BFE9F6000001B40248844601BC98
:103D6000604700BFBD5C010001B40248844601BC4D
:103D7000604700BF6137010001B40248844601BCBE
:103D8000604700BFD544010001B40248844601BC2D
:103D9000604700BFDD3F000001B40248844601BC1B
:103DA000604700BF9573010001B40248844601BC1E
:103DB000604700BFC166010001B40248844601BCEF
:103DC000604700BFE90B010001B40248844601BC12
:103DD000604700BF9D6A000001B40248844601BCF0
:103DE000604700BF8D11010001B40248844601BC48
:103DF000604700BFD1AE000001B40248844601BC58
:103E0000604700BF0534010001B40248844601BC8C
:103E1000604700BFEDA5000001B40248844601BC24
:103E2000604700BFB70E000001B40248844601BCE1
:103E3000604700BF75F8000001B40248844601BC29
:103E4000604700BF1DA2001101B40248844601BCB6
:103E5000604700BF3D71010001B40248844601BCC7
:103E6000604700BF0189000001B40248844601BCDC
:103E7000604700BFC115010001B40248844601BC7F
:103E8000604700BF7912010001B40248844601BCBA
:103E9000604700BFC1A5000001B40248844601BCD0
:103EA000604700BFE917010001B40248844601BC25
:103EB000604700BFA9D8000001B40248844601BC95
:103EC000604700BFED6B010001B40248844601BCAD
:103ED000604700BFE94C010001B40248844601BCC0
:103EE000604700BF5976010001B40248844601BC16
:103EF000604700BFF90D010001B40248844601BCCF
:103F0000604700BF21A9000001B40248844601BCFB
:103F1000604700BFCD0C010001B40248844601BCDB
:103F2000604700BFED68010001B40248844601BC4F
:103F3000604700BF53B9000001B40248844601BC89
:103F4000604700BFE927000001B40248844601BC75
:103F5000604700BF2D6C010001B40248844601BCDB
:103F6000604700BFE512010001B40248844601BC6D
:103F7000604700BF6911010001B40248844601BCDA
:103F8000604700BFF935010001B40248844601BC16
:103F9000604700BFA1B5001101B40248844601BCCE
:103FA000604700BFD9B0000001B40248844601BC9C
:103FB000604700BF75A9000001B40248844601BCF7
:103FC000604700BFF535010001B40248844601BCDA
:103FD000604700BF8512010001B40248844601BC5D
:103FE000604700BF8937010001B40248844601BC24
:103FF000604700BF016C010001B40248844601BC67
:10400000604700BF85C1000001B40248844601BC7E
:10401000604700BFC9A9000001B40248844601BC42
:10402000604700BF0934010001B40248844601BC66
:10403000604700BF19FA000001B40248844601BC81
:08404000604700BF090E0000FB
:104048000200000046BE00110100000058BC00112B
:104058000200000042BE0011010000008840FF1F5E
:104068000200000060BC001101000000C061FF1FD9
:104078000200000040BE0011030000003461FF1F71
:10408800120000000200000046BE001101000000FE
:10409800A0BC00110200000042BE00110100000097
:1040A8009DBC001102000000AABC00110300000022
:1040B8006F61FF1F0200000040BE001103000000F6
:1040C8008461FF1F0200000042BE001101000000D1
:1040D8009CBC001102000000A8BC001103000000F5
:1040E8004561FF1F0200000040BE001103000000F0
:1040F8006661FF1F0200000046BE001101000000BB
:10410800E0BC00110200000042BE001101000000E6
:10411800D141FF1F02000000F2BC001101000000A5
:10412800DBBC00110200000042BE001101000000CB
:10413800D041FF1F02000000F0BC00110100000088
:104148008C61FF1F0200000042BE00110100000048
:10415800CF41FF1F02000000EEBC0011010000006B
:10416800CBBC00110200000042BE0011010000009B
:10417800CE41FF1F02000000ECBC0011010000004E
:10418800C6BC00110200000042BE00110100000080
:10419800CD41FF1F02000000EABC00110100000031
:1041A800C1BC00110200000042BE00110100000065
:1041B800CC41FF1F02000000E8BC00110100000014
:1041C800BCBC001102020202020200000000000052
:1041D8000D0C0000A54B00116B4B001134BD0011F4
:1041E80090011D0018001800FFFF070102030405D5
:1041F80006020106000000000000000000000000A8
:1042080000000000000000000000000000000000A6
:10421800030000000200000046BE0011010000007B
:1042280054BD00110200000042BE00110100000050
:104238008C42FF1F020000005EBD0011010000005B
:10424800BA61FF1F0200000040BE00110300000019
:104258002464FF1F0200000042BE0011010000009C
:104268008C42FF1F020000005CBD0011010000002D
:10427800BC61FF1F0200000040BE001103000000E7
:104288001C64FF1F126C6C6C00000000005800409A
:10429800151600000001000000000111FFFF0000DA
:1042A8005048593600000000000000000B000500CF
:1042B800F0000000B4000028002800283075A00095
:1042C800A000A000A00000080008E001F000100015
:1042D8001000100010001000100050005000500096
:1042E80010001000D0070000000000000F000100BF
:1042F8000500307507001000010081FF0000000074
:10430800FF000000057400110D7200119D6F00116F
:10431800FFFF0100FF000000219E00119D9B00117E
:10432800B59A00110000000000000000000008001D
:10433800040000003B0001085902E0018821280020
:10434800FF0000000200000046BE0011010000004E
:104358000CBF00110200000042BE00110100000065
:10436800C943FF1F020000003EBE0011010000000B
:10437800F067FF1F0200000042BE001101000000AC
:10438800C843FF1F020000003CBE001101000000EE
:10439800C643FF1F0200000042BE001101000000DA
:1043A800C443FF1F020000003ABE001101000000D4
:1043B800BC43FF1F180018001D00900102000003F5
:1043C800020200000200000046BE001101000000C9
:1043D80020BF00110200000042BE001101000000D1
:1043E8000C44FF1F0200000038BE0011000000004E
:1043F800000000000200000040BE001103000000A1
:064408001068FF1F20FFF9
:040000051FFF184180
:00000001FF
